:0200000260009C
:10400000000001205D4306004543060047430600CB
:10401000494306004B4306004D43060000000000E4
:104020000000000000000000000000004F430600F8
:1040300051430600000000005343060055430600AC
:104040005743060057430600616A060057430600BF
:1040500057430600574306005743060057430600E0
:1040600057430600574306005743060057430600D0
:1040700057430600574306005743060057430600C0
:10408000ED910600574306005743060057430600CC
:1040900057430600574306005743060057430600A0
:1040A0005743060057430600574306005743060090
:1040B00057430600574306000000000000000000C0
:1040C0005743060057430600574306005743060070
:1040D000518B0600574306005743060000000000BE
:1040E00000000000000000000000000000000000D0
:1040F00000000000000000000000000000000000C0
:1041000000000000000000000000000000000000AF
:10411000000000000000000000000000000000009F
:10412000000000000000000000000000000000008F
:10413000000000000000000000000000000000007F
:10414000000000000000000000000000000000006F
:10415000000000000000000000000000000000005F
:10416000000000000000000000000000000000004F
:10417000000000000000000000000000000000003F
:10418000000000000000000000000000000000002F
:10419000000000000000000000000000000000001F
:1041A000000000000000000000000000000000000F
:1041B00000000000000000000000000000000000FF
:1041C00000000000000000000000000000000000EF
:1041D00000000000000000000000000000000000DF
:1041E00000000000000000000000000000000000CF
:1041F00000000000000000000000000000000000BF
:10420000314932480A1A02D0072291438D4630497B
:1042100030480A1A06D00722914381F30988022206
:1042200082F314882C482D492D4A00F03CF82D4883
:104230002D492E4A00F037F82D482E492E4A00F01D
:1042400032F82E482E492F4A00F02DF82E482F49DB
:104250002F4A00F028F82F482F49304A00F023F861
:104260002F483049304A00F01EF8304830490022CB
:1042700000F024F82F483049002200F01FF82F4AA0
:1042800090471F481F49884205D00268043003B494
:10429000904703BCF7E700208646EC46002000214B
:1042A000274A9047FEE7884207D0521A05D0037884
:1042B00001300B700131013AF9D17047884202D0C8
:1042C00002700130FAE770470000012000F800207A
:1042D0000000012000000120F8F206001C00002070
:1042E00078000020B8430600B843060040BD060031
:1042F000F8F206001C0000201C000020FCBD060097
:10430000FCBD0600FCBD0600FCBD0600FCBD0600B1
:10431000FCBD0600FCBD0600FCBD0600F6F2060072
:1043200054F3060078000020780000207800002078
:10433000F0370020F0370020F037002085430600DA
:10434000E5740600FEE7FEE7FEE7FEE7FEE7FEE7B0
:10435000FEE7FEE7FEE7FEE700F002B8FFF7FCBF6E
:104360000F484FF00701884385460E4880470E48A6
:10437000016841F470010160BFF34F8FBFF36F8F8D
:10438000FFF73EBF09480A490A4A884207D0521A35
:1043900005D0037801300B700131013AF9D1704733
:1043A00000000120F992060088ED00E0E8BD06005B
:0843B000080000201C000020A1
:1043B8007047000007B5044B0093044A402300F0FF
:1043C80032F803B05DF804FBD943060079000020F9
:1043D8002DE9F84388461446B2B10F4B0F4E03251A
:1043E800002743F00109224608EB0701002007F0E7
:1043F8002FFB0744241A48B933782BB14FF47A407D
:10440800C847013D02D13570BDE8F88301233370F8
:10441800002CE8D1F8E700BF00BE060078000020B5
:10442800704707F045BBF0B595B01D4616460846DF
:104438000C4602F02EF81A9B0D93CDE9086500256D
:104448002B46082205A920460A958DF82C500C9574
:1044580002F046F8079B0293069B03939DF81430DD
:104468008DF8115003F00302012A1DD1BDF8142064
:10447800059DC3F3C203C2F383168DF81030B20052
:1044880008230EA9204602F02BF8C5F3952508ABA2
:104498000093324602AB0EA9284600F0D5FB204611
:1044A80001F0FBFF15B0F0BD022AF8D1BDF8165097
:1044B800C3F3C203C5F389158DF810300827082DFA
:1044C8002E4628BF08263B4632460EA9204602F053
:1044D80007F8AD1B08AB02AA31460EA8374400F016
:1044E80017FC002DEBD1DAE708B5FFF79AFF07486C
:1044F800042100F015FB002803DA0549412001F0EA
:10450800DDFA044B01225A7108BD00BFD8BD060070
:1045180014BE06001C000020037813F0040216D015
:1045280003F00303012B03D0022B09D001207047AD
:104538000A6800880232C0F3831002440A60F5E773
:104548000B684288023303EB92130B60EEE71046C8
:10455800704700002DE9F04FDFF828A10F4685B01D
:104568000446861C0020154601F06CFADAF804208F
:104578003A60DAF80830414F03F580639B1AA7F1D7
:104588000409A7F10808B3421AD30020002D71D0FE
:1045980004F00F039B0143F0050363F30F00DAF8FF
:1045A8000430C3F30902033233444AF822000020DE
:1045B800CAF8043001F056FA012005B0BDE8F08FC2
:1045C8000121384601F0C1FA484601F0D9FA4046BF
:1045D80001F0D6FADAF808000090C0F309000330B9
:1045E8000AEB80006946FFF797FF009B8346C8B92E
:1045F800C3F309020AEB8202D16801919A1C0133C4
:10460800C3F309030AEB83030092D86801F003039C
:10461800012B27D0022B08D019494FF4C27001F0A2
:104628004DFA0CE0C3F30900D9E7BDF80630C3F32F
:10463800891303334FEA104B02EB93030093404670
:1046480001F0A1FA10B1009BCAF808305946384663
:1046580001F07BFADAF80830DAF8042003F5806311
:104668009B1A90E7BDF80430C3F383134FEA104B4D
:104678001344E3E7A40544F0060090E7A8110020DE
:10468800B5BE06008C010020064B074810B5002275
:104698001A7001F0B7FE044610B9044801F034FF5F
:1046A800204610BD8C010020B0BD060054BF060096
:1046B80030B50A4C71B10A4A0A49121BD2080023C4
:1046C8009A4201D1002030BD31F82350854202D0F2
:1046D8000133F5E7034654F83300F4E748BD060014
:1046E800B0BD06001C000020094B013903EBC000D7
:1046F800032909D8DFE801F00A02040604207047FC
:104708000079704740797047002070470220704751
:1047180048BD0600034BD3E90130C31A584258413B
:10472800704700BF8C0100202DE9F04385B0FFF7EA
:10473800F1FF0646002840F0EC80774C04F58055E0
:10474800A861BFF34F8FA3680093C3F30903033332
:1047580004EB83006946FFF7DFFE009B10B1AA69EE
:10476800002A5DD0C3F30902991C013304EB8202CD
:10477800C3F3090304EB8303D268DB68029302F0F6
:104788000303022B0192009155D1BDF8063063480E
:10479800C3F389184746502F28BF502707F108014F
:1047A80067F38F13C1F30901ADF8063001F042FE3B
:1047B8000646002800F0998001F06BFE00230822CD
:1047C80001A9304601F078FE0099CB43C3F30903F1
:1047D8000133C1F309010331B7EB830F4FEA8302B9
:1047E80004EB810124D95FFA82F90823A7EB0907B2
:1047F800304601F061FEFFB209F10803484903F0B1
:10480800FC033A46304601F057FE009B08F10308C6
:1048180003EB98030093AB69002B43D12F6954E055
:1048280062689A4291D8A260304605B0BDE8F0832C
:1048380008233A46E6E7012B57D1BDF8043037483C
:10484800C3F38311062928BF062161F389130231B6
:1048580001F00F018900ADF8043001F0EBFD0646C8
:10486800002842D001F015FE0023082201A9304695
:1048780001F022FE0027BDF80420C2F38312BB001A
:10488800974203F10803C6D200994A1CC1F30901F3
:104898000331009204EB81010422304601F00CFE42
:1048A8000137E8E7304601F0F8FDFFF733FF80F005
:1048B8000100C6B2B8E7FB685B7923B13B683146B3
:1048C8001B6838469847FB681F68002FF3D13046AD
:1048D80001F0E3FD384601F0B5F8AB690BB9009B70
:1048E800A360002001F0BEF8DFE72C6954B90D4B36
:1048F8000D480E49C01AC008000440F0020000F03C
:1049080073F8D2E7236820469B689847E3681C68D9
:10491800ECE7002688E700BF8C010020B0BD060048
:104928009801002048BD060058BD06003EBF06009D
:104938002DE9F34704460F46914601A9012218467E
:104948001E46FFF707FEDFF89C8078B3019D002321
:10495800A81CB34203EB000132D11E48002101F02C
:10496800B9F880F3100A1C4B1C4A4FEA14499B1AE9
:10497800B9EBD30F04D31A4940F2A91001F09EF8FD
:104988006B1CC3F30903E40008EB830304F0380449
:1049980049EA0A40C5F3090544F00104D860033523
:1049A80044EA861343EA872348F8253098F800300C
:1049B8001BB1FFF7B9FE0028FBD102B0BDE8F087B4
:1049C800C1F3090108EB810159F82320CA600133BA
:1049D800BFE700BFA8110020B0BD060048BD060013
:1049E800B5BE06008C01002000231A46FFF7A0BFC1
:1049F80007B50123019201AAFFF79AFF03B05DF8FA
:104A080004FB07B5CDE9002302236A46FFF790FFB0
:104A180003B05DF804FB1FB5CDE90123069B0393A2
:104A280001AA0323FFF784FF05B05DF804FB1FB557
:104A3800CDE90023069B0293079B03936A46042350
:104A4800FFF776FF05B05DF804FB7FB5CDE90123DC
:104A5800089B0393099B04930A9B059301AA0523CA
:104A6800FFF766FF07B05DF804FB00002DE9F74388
:104A78000446D01C8846164601A900228008FFF784
:104A880069FD254D98B3019FB81C0190C0F309003A
:104A9800C0F58063B6EB830F00F103004FEA83098A
:104AA80005EB80002CD83246414607F097F81B48A2
:104AB800002101F00FF880F310007B1CC3F30903F9
:104AC800C7F30907220C05EB8303033742EA0040CA
:104AD800E400D86004F0380455F8273044F00204A4
:104AE80044EA865203F47C131A4345F827202B78AE
:104AF8001BB1FFF719FE0028FBD103B0BDE8F08316
:104B08004A46414607F06AF8A6EB090208EB090194
:104B180005F10C00C9E700BF8C010020A811002096
:104B280030B50E4C226903460020114629B9D968D0
:104B3800087142B923610A6030BDC9680D798542A0
:104B480006D00968F2E7D26814680C601360F3E7CE
:104B580001300A28E9D14FF0FF30EDE78C11002031
:104B680038B5084B03F58052012514691D7004B946
:104B780038BDE3685D71236820465B689847E36841
:104B88001C68F4E78C01002030B5C38885B0044662
:104B98000D4633B1144A00921449154A284601F0CB
:104BA80095F8217A05291DD0637A4BB1A088FFF7C3
:104BB8009BFD104B104953F82020284601F086F839
:104BC800227A0E4BA08853F8222003920021FFF787
:104BD8006FFD039A0A490346284605B0BDE83040F0
:104BE80001F074B805B030BD80BF060068BF06008C
:104BF80060BF0600F0BF0600D5EB060014C0060033
:104C080085BF060007B503460846197A052911D05D
:104C18005B7A2BB1094A0A49019001F057F80198CB
:104C28000849019001F052F8019803B05DF804EBCF
:104C380001F03AB8002AF8D0F2E700BF80BF0600BA
:104C4800D5EB06007DBF06002DE9F04385B01F4671
:104C58000C9D002395F80C902B7306460C46904645
:104C680029463846FFF790FFB8F1060F09D8DFE864
:104C780008F00412181F283340003146284601F076
:104C880025F8002229463846FFF7BCFF85F80C9026
:104C980005B0BDE8F08322683146284601F016F8D1
:104CA800EFE7D4E900233146284601F00FF8E8E79A
:104CB800A36800933146D4E90023284601F006F89A
:104CC800DFE7E3680193A36800933146D4E9002342
:104CD800284600F0FBFFD4E723690293E3680193B9
:104CE800A36800933146D4E90023284600F0EEFF7C
:104CF800C7E76369039323690293E3680193A36891
:104D080000933146D4E90023284600F0DFFFB8E7D6
:104D180008292DE9F74F80460E4617461C463DD810
:104D280000251B7B2573214610460193FFF72CFFB6
:104D3800DFF88CA0DFF88CB0AE4232D918F8052025
:104D48005946204600F0C2FF0135082DF4D11B4911
:104D5800DFF874A0DFF874B0204600F0B7FF4FF01A
:104D680000094E4524D918F809507E2D1ED828462A
:104D780006F0F8FE002814BF2A462E22594620467F
:104D880000F0A4FF09F10109B9F1080FE9D10122E6
:104D980021463846FFF736FF019B237303B0BDE871
:104DA800F08F5146204600F091FFCDE72E22E5E72F
:104DB8005146204600F08AFFE4E700BF99BF06008D
:104DC80095BF06008FBF060097BF06009BBF060071
:104DD80008B543090CBF4FF0FF33002300F01F0054
:104DE80023FA00F0C30704D403494FF4F67000F027
:104DF80065FE4FF0A04008BD28C00600032810B586
:104E0800044603D90649412000F058FE054B1C5DB5
:104E18002046FFF7DDFF0123A340C0F80C3510BD85
:104E280053C00600C7C00600032810B5044603D9BE
:104E38000649472000F042FE054B1C5D2046FFF75F
:104E4800C7FF0123A340C0F8083510BD53C00600B2
:104E5800C7C0060008B50020FFF7E6FF0120FFF7EE
:104E6800E3FF0220FFF7E0FFBDE808400320FFF75B
:104E7800DBBFC20738B5044616D51120FFF7A8FFD7
:104E88000325C0F844571220FFF7A2FFC0F848577F
:104E98001320FFF79DFFC0F84C571420FFF798FF29
:104EA800C0F85057FFF7D6FFA30714D50D20FFF71A
:104EB8008FFF0C24C0F834470E20FFF789FFC0F895
:104EC80038470F20FFF784FFC0F83C471020FFF752
:104ED8007FFFC0F8404738BD43689B68184708B54E
:104EE800436808305A7902F06FFA002008BD2DE9AE
:104EF800F0410C469CB008461F460392FFF7ECFFB2
:104F0800D4F80480039998F80550BD4228BF3D465F
:104F180006462A4604A802F03BFA98F8052022998A
:104F28000CA802F051FA00960CAB2A4604A904F129
:104F3800080003F07FF9002848F2425018BF00200B
:104F48001CB0BDE8F0810023C0E902328B881A4406
:104F5800B1F9063002611A44C0E9001142610888BB
:104F6800003818BF012070474268118838B50346D9
:104F7800002937D0148A02F1100141602CB9C268A7
:104F88000168FFF7E0FF204638BD9078118900F0EE
:104F98003005302D14D1947C04F03004302C1BD112
:104FA80090881969091A19610021908AB2F91620A6
:104FB8000844196901441961114459610120E3E762
:104FC80000F0F004202C07D150894143002DECD18A
:104FD800986801309860E8E700F0C000802808BFB2
:104FE8000421F3E70846CFE770B5466804460D4646
:104FF80063681A88AA4204D19B7803F00F03082B30
:1050080007D12046FFF7B0FF6368B342F0D1002014
:1050180070BD0120FCE743681A44426011B10139B0
:105028009A4201D10120704713F8010B01F8010FD2
:10503800F6E770B54568AA7802F00F06082E86B024
:1050480003461FD103691C6800260CB906B070BD61
:10505800236862689D68267329466846FFF773FFD0
:105068006368049304F10C030593AB7803F0C00361
:10507800802B08BF231D684608BF0493FFF7D9FF9C
:10508800A468E2E712F0C00122D102F03000102833
:105098000CD15A691170072EEC6818690BD10146BA
:1050A800204606B0BDE8704000F01AB89006F2D568
:1050B8005B691980CAE72A89214624B106B0BDE890
:1050C800704006F08BBD06B0BDE8704006F0AFBD7D
:1050D8008029BBD10069002192060160B6D5E7E7B7
:1050E8007FB50A4601466846FFF72DFF30B168468E
:1050F800FFF79FFF6846FFF737FFF7E707B05DF850
:1051080004FB836810B504460BB9002010BD036882
:10511800012298470028F8D0A368013BA360F5E76F
:105128002DE9F3410F460DF107018046FFF7E9FF2E
:10513800054620B90025284602B0BDE8F0819DF952
:1051480007309DF80740002B13DA04F07F04072688
:105158000DF107014046FFF7D4FF0028EAD09DF87B
:10516800072002F07F03B3401C43130606F107062D
:1051780001D43C60DFE7232EEAD1DBE730B50446F3
:1051880085B01546A9B90268114B9A4211D0102D65
:1051980006D82A4669462046FFF7F0FF05B030BD1D
:1051A800102269462046FFF7E9FF0028F6D0103D97
:1051B800EDE7A368AB4201D20020EFE723682A4657
:1051C800204698470028F7D0A268521BA260E5E75E
:1051D8001F500600F7B50E4601A907461546FFF70A
:1051E8009FFFA0B1019A511C4FF0000404D2B3787C
:1051F80003F0C003802B01D1204608E033898B429D
:10520800FAD329463846FFF7B9FF019BEC5403B09F
:10521800F0BD73B50D4601A906461446FFF780FF99
:1052280098B1019AB2F5803F11D2AB7803F0C00370
:10523800802B02F102010AD02B898B4207D3214629
:10524800304621F8022BFFF799FF02B070BD00200D
:10525800FBE7000010B5034C82600022C0E9004162
:10526800C26010BD1F5006002DE9F341002580469D
:105278000E462F462C460DF107014046FFF741FF29
:10528800C0B19DF807C0A4F120030CF07F02C4F15F
:10529800200102FA03F322FA01F10B43A2401CF0A9
:1052A800800F45EA020547EA030704F1070404D121
:1052B800C6E9005702B0BDE8F081462CDBD10020DA
:1052C800F8E737B50D4669461446FFF7CDFF70B1CC
:1052D8002B89082B0DD1DDE90032C4E90032DDE964
:1052E8000001914208BF98420CBF0120002003B082
:1052F80030BD042B03D1009B23600022EFE7022B73
:1053080003D1009B23809BB2F7E7012B04D1009BBC
:10531800237003F0FF03F0E70020E8E737B50D46F8
:1053280069461446FFF7A0FF30B12B89082BDDE949
:10533800001203D1C4E9001203B030BD042B4FEAB8
:10534800E17009D121600B460246824208BF8B42B8
:105358000CBF01200020EFE7022B03D10BB2238002
:10536800DA17F2E7012B02D14BB22370F8E70020DD
:10537800E2E7F7B51F4600233B700D460B7013603C
:1053880001A904461646FFF7CBFE30B9A36813B946
:1053980001233B70002003B0F0BD019C002CF7D026
:1053A800E30804F0070433602C70F4E713B50446EF
:1053B800052925D8DFE801F0030F1724242201224C
:1053C80001A92046FFF7DAFE18B19DF90430002B39
:1053D800F5DB02B010BD08220021204602B0BDE86E
:1053E8001040FFF7CBBE01A9FFF79AFE0028F0D0C6
:1053F800019A00212046FFF7C1FEEAE70422EBE705
:105408000020E6E773B50D4601A90446FFF788FEBC
:10541800064618B90026304602B070BD94E80F0061
:1054280085E80F0001998A42F4D3A960A3685B1A42
:10543800A360F0E72DE9F0435668B37813F0C00491
:1054480089B007468C46154603D0402C69D0002405
:105458000CE003F00F02604903F03003202B51F8F1
:10546800228025D006D8E3B1102B17D0204609B0EA
:10547800BDE8F083302BF9D16B6931881980072A90
:1054880009D121463289286906F0D1FB6B68296960
:10549800D868FFF725FE2A69696840E06B69012230
:1054A8001A702A693146434609B0BDE8F0431847E7
:1054B800BCF1020FD5F8149024D1042A22D804A9EB
:1054C800FFF7A0FF04460028C1D0069B2BB16968EE
:1054D800B9F800304A899A4205D8059B7B60069B3B
:1054E800002BC3D0B3E708892A6903FB002204A86C
:1054F800C04728B1B9F800300133A9F80030E4E713
:105508000446EAE7B9F8003072899A429FD931898E
:105518002A69581C03FB0122A9F8000031463846C5
:10552800C1E7D2F81080464656F8043B23B909B0C3
:10553800BDE8F043FFF73ABF022914D104A9FFF7E9
:1055480061FF002883D0D8F800306968324604A883
:105558009847044600283FF47AAF069B002BF2D107
:10556800059B7B6082E7012926D005292CD00029DC
:105578007FF46DAF0C460DF1040901340B2C3FF498
:1055880066AF012249463846FFF7F8FD00283FF488
:105598005EAF19F9013B002BEFDB104B049301AB15
:1055A800CDE90534002307936968D8F800303246FE
:1055B80004A89847044659E7082201A9FFF7DEFD29
:1055C80008240028E9D142E704220DEB0201FFF785
:1055D800D5FD0424F5E700BFD8C006001F5006001B
:1055E8002DE9F04F91B00446002604A8CDE90266E3
:1055F800FFF7A9FCA3683BBBDDE9053404A89D7847
:10560800FFF7B2FC0028F7D115F0300F03D1059B46
:105618001B8803B10134002C00F0A980630902A99A
:105628000022934240F09C8010AA02EB830304F00E
:105638001F0453F8383CC4F120044FF0FF30E04019
:10564800C31A584258410DE00DF1030301AA0DF1A8
:1056580002012046FFF78DFE38B99DF80330002B74
:10566800CAD1002011B0BDE8F08F019904A8FFF756
:10567800BBFC002850D1019BB3427DD3059D059A00
:10568800937803F00F03082B7FD004A8FFF76CFC76
:10569800059B9D42F3D14FF0FF36019FB7426BD374
:1056A800089B9DF802A0D4F808801D684FF00109F6
:1056B800A368002D5DD098459CD12B68D3F800B025
:1056C800BBF1000F08D053463A4629462046D84732
:1056D8000028C6D0AD68EBE7D3F808B0BBF80030B7
:1056E8009F42F7D16A6859460AA8FFF72CFC6B68F5
:1056F8000E9305F10C030F939BF8023003F0C003DF
:10570800802B04BF2B1D0E930AAA85F80C905146D6
:105718002046FFF78FFEDBE7059B9B7813F0300FE1
:105728000FD1069A3F2A0CD8510910AB03EB81011F
:1057380002F01F020123934051F8382C134341F81B
:10574800383CE5682DB19DF80220019904AB20464C
:10575800A8479DF8021004AA2046FFF76BFE10E048
:1057680051F8045B01357FF47DAF013259E7012020
:1057780078E798457FF43EAF9DF802102046FFF782
:1057880015FE00287FF436AF6BE7168885E737B536
:105798000C460546114620460192FFF7A1FC019AE6
:1057A8002146284603B0BDE83040FFF719BF70B561
:1057B80086B0CE6801920C4602A90546FFF722FE84
:1057C80068B1E06858B1A378019A03F03003202B40
:1057D800314602A805D1FFF7DAFF039B6B6006B0DC
:1057E80070BDFFF7FDFEF8E713B50C466946FFF7F5
:1057F8003BFD60B1DDE900134A0842EAC372C907FC
:105808004FEA530344BFD243DB43C4E9002302B049
:1058180010BD37B50D4669461446FFF7E5FF70B170
:105828002B89082B0DD1DDE90032C4E90032DDE90E
:105838000001914208BF98420CBF0120002003B02C
:1058480030BD042B03D1009B2360DA17EFE7022B4E
:1058580003D1BDF900302380F7E7012B03D19DF96F
:1058680000302370F1E70020E9E713B504220C4665
:105878000DEB0201FFF782FC08B1019B236002B027
:1058880010BD1146FFF7F1BF13B508220C46694653
:10589800FFF774FC18B1DDE90023C4E9002302B066
:1058A80010BD1146FFF7F0BF4B1C30B5DB000446B6
:1058B80012F003009BB20DD1074D2A601A44074B22
:1058C8001A60074B1870074B1870074B1C80074B62
:1058D800198030BD0720FCE74C1200204812002038
:1058E80044120020541200205012002052120020AE
:1058F8002DE9F843DFF8AC80B8F800308B42064653
:105908000D46174640D3002000F09CF8204B214A52
:105918002148197800881478E3B2844238BF0133EB
:10592800C9B234BFDBB20023994226D0147811786B
:10593800CBB2884286BF0133DBB20023137000204C
:1059480000F090F84FF6FF739C421FD0134B1B6872
:1059580043F8347003EBC40996B18DB1104BB8F815
:1059680000001B682A46314604FB003006F036F971
:10597800A9F804500020BDE8F8834FF6FF74DEE76D
:105988000020A9F80400F6E70920F4E70420F2E76C
:105998005412002044120020521200204C12002001
:1059A800481200205012002070B5104C104D22787B
:1059B8002B789A4200D170BD0E480F4A237812689E
:1059C80006880E4802EBC301006852F83320898824
:1059D80003FB060090470A4922780988D3B291420E
:1059E80086BF0133DBB200232370E0E754120020A6
:1059F80044120020501200204C12002048120020AF
:105A08005212002072B6024A1368013313607047BD
:105A180058120020034A1368013B136003B962B6A9
:105A2800704700BF58120020EFF30583C3F3080343
:105A38002BB9EFF31480C04300F001007047012038
:105A48007047000008B5FFF7EFFF012803D00449AD
:105A5800432000F033F8BDE80840FFF7D3BF00BF8C
:105A6800FCC0060008B5FFF7DFFF012803D0044992
:105A7800512000F023F8BDE80840FFF7CBBF00BF76
:105A8800FCC0060030B53AB11368DB430A4D014447
:105A9800814204D1D84330BD4FF0FF33F6E710F808
:105AA800012B5340082213F0010418BF2C46013A79
:105AB80084EA5303F7D1EBE72083B8ED07B5CDE9C6
:105AC80000016A46002144F2020001F0DDFC03B047
:105AD8005DF804FB10B5034653E8000F0A4643E897
:105AE800002494F0000FF7D110BD10B5034653E819
:105AF800000F40EA010243E8002494F0000FF6D1B9
:105B080010BD10B5034653E8002F42EA010043E8F0
:105B1800000494F0000FF6D110BD10B5034653E809
:105B2800000F00EA010243E8002494F0000FF6D1C8
:105B380010BD10B5034653E8002F02EA010043E800
:105B4800000494F0000FF6D110BD10B5034653E8D9
:105B5800002F02EB010043E8000494F0000FF6D197
:105B680010BD10B5034653E8002FA2EB010043E82F
:105B7800000494F0000FF6D110BD0121FFF7B5BF66
:105B88000121FFF7BEBF0021FFF7C7BF0021FFF7C4
:105B9800D0BF000010B50446002834D003681BB9F4
:105BA8001A49FF20FFF78AFF636823B917494FF4A2
:105BB8008070FFF783FFA36823B9144940F20110EE
:105BC800FFF77CFFE36823B910494FF48170FFF7B2
:105BD80075FF238A23B90D4940F20310FFF76EFFC2
:105BE800D4E9012321689B1ADBB20A60013BDBB2CE
:105BF800FF2B226802D10020107110BD1168481CCB
:105C080010600B70F2E70E20F7E700BF8CC10600AA
:105C180038B5044620B911494FF49270FFF74EFF8A
:105C28000020FFF70FFF226863681168994213D9B3
:105C3800481E106011F8013CE568218A01FB0355F4
:105C4800A36811791B1ADBB2994200D213710020A4
:105C5800FFF708FF284638BD0025F8E78CC1060085
:105C680038B50C46054620B90E4940F24710FFF7F3
:105C780025FF24B90B494FF4A470FFF71FFF00203C
:105C8800FFF7E0FE2A681368591C1160E968641A76
:105C9800298AB4FBF1F41C70BDE838400020FFF7F6
:105CA800E1BE00BF8CC1060010B5044618B906490C
:105CB8003120FFF703FFA2682AB1636921682069D0
:105CC80098470023A36010BD0EC206000EB433B57A
:105CD800059D044618B911494220FFF7EFFE636994
:105CE8001BB90E494320FFF7E9FE23681BB90B498E
:105CF8004420FFF7E3FE63681BB908494520FFF716
:105D0800DDFE35B106AB01AA29462046019300F015
:105D180079F802B0BDE8304003B070470EC2060003
:105D28000A2938B504460D4602D10D21FFF7F8FFC0
:105D3800A3682268591CA160D554D4E901329A425B
:105D480004D32046BDE83840FFF7AEBF38BD000099
:105D58002DE9F84F9846DDE90A43154682460F4675
:105D68000A464FF00109AA420FD2C14538BFC146C1
:105D780013F0010B01D16CB900240126B8F1010F11
:105D88001BD908F1FF386E43F8E709F10109B2FBA6
:105D9800F5F2E8E79B070ED5B8F1000F0CBF3026E7
:105DA8002026A145E9D2013C31465046FFF7B8FF0D
:105DB800002CF6D1E0E72026F3E7B7FBF6F39D4287
:105DC800E1D9DFF83C80B7FBF6F3504618F803102A
:105DD80006FB1377FFF7A4FF3346AB42B6FBF5F695
:105DE800F1D2BBF1000F02D00CB1A14501D3BDE83F
:105DF800F88F20215046013CFFF792FFF4E700BFDF
:105E080005C306002DE9F74F88461746054620B911
:105E1800AF4940F25220FFF751FE6B6923B9AC49F4
:105E28004FF41570FFF74AFE2B6823B9A84940F2D2
:105E38005520FFF743FE6B6823B9A54940F2562069
:105E4800FFF73CFEB8F1000F00F03E8118F8011B87
:105E580049B92B7B002B00F03781284603B0BDE8F9
:105E6800F04FFFF721BF252940F0B780002698F8AA
:105E780000302D2B424608F1010823D0302B24D0C6
:105E88002B2B25D000242A2B02F1010123D13B68BA
:105E98001A1D1B683A601C440A4613782E2B26D11B
:105EA80001324FF0000A104610F8011BA1F1300C26
:105EB800BCF1090F1DD80A2303FB0A13A3F1300A0A
:105EC8000246F0E746F00106D1E746F00206CEE7C3
:105ED80046F00406CBE711F8013CA3F1300009288D
:105EE800DBD80A2202FB0434303C0A46CBE74FF0E9
:105EF800000A12F8011B01F0FB0068289046F8D050
:105F0800782909D86F290CD8632962D022D8252985
:105F180063D0582900F0888098F80030002B95D17C
:105F280097E770390829F7D801A353F821F000BF83
:105F3800AB600600215F0600215F06004160060095
:105F4800215F06001F600600215F0600215F060032
:105F580031600600642901D06929DDD13A68D2F898
:105F68000090111D89EAE9723960A2EBE9724FF0DD
:105F7800010B092A35DCD34538BFD3462CB1B9F11A
:105F8800000F01DB720700D5013CB30702D5BAF157
:105F9800000F03D0F00701D44CBB0024B9F1000F67
:105FA8002DDAC9F100092D212846FFF7B9FE06F0C0
:105FB8000302022A04D1BAF1000F01D11CBB00244C
:105FC800CDE9004653460A2249462846FFF7C0FE57
:105FD800A2E73B681A1D19783A602846FFF7A0FE29
:105FE8009AE70A230BF1010BB2FBF3F2C1E7A345D1
:105FF800D4D220212846013CFFF792FECCE7710756
:10600800D5D52B21D0E7A345DAD230212846013C4B
:10601800FFF786FED2E73968CDE900460A1D3A60E7
:1060280053460A220968D0E739680A1D3A60CDE963
:10603800004653461022F5E73B681A1D3A6016F0F1
:106048000106D3F8009024D1B9F1000F03D04846D7
:1060580005F042FE0646B4421DD809F1FF3919F889
:10606800011F00293FF458AF2846FFF759FEF6E70D
:1060780028460136FFF754FE19F806100029F7D113
:10608800A642BFF449AF20212846013CFFF748FE4D
:10609800F6E70026F0E720212846013CFFF740FEFE
:1060A800D9E73B681A1D3A60302128461C68FFF77B
:1060B80037FE78212846FFF733FE00220823CDE972
:1060C80000322146102280E703B0BDE8F08F00BF00
:1060D80086C2060070B50D461646044618B908492A
:1060E8005520FFF7EBFC1DB905495620FFF7E6FCE4
:1060F8002B68256031462046BDE87040184700BF30
:1061080015C306002DE9F041DDF818800E46174644
:106118001D46044618B922498820FFF7CFFC1FB94D
:106128001F498920FFF7CAFC23681BB91C498A202C
:10613800FFF7C4FC45BB1A498B20FFF7BFFCB20729
:1061480003D017499120FFF7B9FCBB0703D01449C6
:106158009220FFF7B3FCE3689E4204D322696B1ECA
:106168003344934203D90E499320FFF7A7FC2368D1
:10617800CDF81880D3F80CE03A462B463146204635
:10618800F446BDE8F041604763685A68B5FBF2F32E
:1061980002FB1353002BD2D001498E20CDE700BF5C
:1061A80015C306002DE9F0410D4616461F46044664
:1061B80018B919499E20FFF781FC23681BB91649B5
:1061C8009F20FFF77BFC1EB91349A020FFF776FC40
:1061D80063681B68013B2B4203D00F49A320FFF7DC
:1061E8006DFCE3689D4207D363681A686B1E02FB67
:1061F80006332269934203D90749A520FFF75EFCBD
:106208002368D3F810E032463B4629462046F44638
:10621800BDE8F041604700BF15C3060070B550B92E
:106228000E4D0F4C0026641B1423B4FBF3F4B44248
:1062380008D1002010E00368002BF1D0BDE87040C1
:10624800DB6918472B6813B901361435EFE7DB69AA
:10625800284698470028F7D070BD00BF08000020E6
:106268001C000020014B436000207047A8C30600B3
:106278000846704700207047024B1868003818BF5E
:10628800012070475C12002008B50248FFF77EFC29
:10629800002008BD5C12002008B510461A4605F01B
:1062A8009DFC002008BD00002DE9F041804686B025
:1062B80011480F4616461D46FFF75FFC0446C8B94D
:1062C800AA083146384600F0A7FB0B48FFF75EFCEA
:1062D800D8F8083053B101228DF800200C9A0592A5
:1062E800CDE90147CDE9036568469847204606B0E1
:1062F800BDE8F0811124F9E75C1200202DE9F04394
:10630800814687B014480E4615469846FFF735FC77
:106318000446F0B90746BD4215D10F48FFF736FCD1
:10632800D9F808305BB102228DF800200022CDE9AF
:106338000126CDE90325CDF8148068469847204604
:1063480007B0BDE8F08306EB073000F037FB0137F4
:10635800E1E71124F3E700BF5C1200202DE9F74FB5
:1063680099469DF83030009388469346064618B9FA
:106378002349B620FFF7A2FBF28871794A43043A11
:106388004A4505D81E490192C420FFF797FB019A98
:10639800DBF80070B6F806A007EB0901914209F195
:1063A800040488BFA2EB0907B4FBFAF5CBF8007028
:1063B8000AFB154445B9AAEB040BBB4528BFBB46ED
:1063C8002FB903B0BDE8F08F3668013DF2E7009BB6
:1063D800043408EB050034445A466BB12146A7EB58
:1063E8000B0705F0FBFBBA455D443668D3464FF012
:1063F800000428BFBB46E3E701462046EFE700BF9D
:10640800D4C30600FFF7C6BBF8B546790146721E2D
:106418000546002393422D6803D30024A64202D8E0
:10642800F8BD0133F6E70F682846FFF719FC013479
:106438003946F3E72DE9F843068ACD1C0746FFF7EE
:10644800E7FB043E35440446B5FBF6F5F0B14FF4DE
:106458008073EDB28380C680013D076081464FF0AE
:106468000008A84512D23846FFF7D2FB064648B1C5
:1064780063790133637108F10108C9F80000076006
:106488008146EEE72046FFF7BFFF34462046BDE8C9
:10649800F88301210430FFF758BB10B501210446E9
:1064A8000430FFF75EFBC0B220B92046BDE81040BB
:1064B800FFF7AABF10BD00001FB5144603920022C3
:1064C800009203AAFFF74AFF039BA34203D00349A4
:1064D800F620FFF7F3FA04B010BD00BFD4C30600DE
:1064E8001FB5144603920122009203AAFFF736FF54
:1064F800039BA34204D003494FF48070FFF7DEFAF0
:1065080004B010BDD4C30600836800225A60C3E9F2
:1065180004229A60DA601A607047000010B50D49CD
:10652800A1F58C72914201D800200FE08C1AE30F7C
:1065380003EBE4035B1002EBC30452F833308342ED
:1065480005D802D204F10802ECE7606810BD2146C4
:10655800E8E700BF14C9060008B5FFF7DFFF024BE4
:10656800002808BF184608BDE7C706002DE9F04F08
:10657800C9B008AA01F1400514464B780E781B04EF
:1065880043EA0663CE7833438E78043143EA062320
:106598008D4244F8043BF0D11024916B16464FEA23
:1065A800F14383EA714383EA9123716A366852F8AA
:1065B800045F31440B444FEAB54181EAF51181EAA1
:1065C800D50101340B44402CD363E6D1D0E914E360
:1065D8000093836D0193C36D0293036E0393436E1F
:1065E8000493836E0593C36E0693DDE9057BDDE9AD
:1065F800031CDDE901592B4B009E079374464FF0AD
:106608000008079B53F8042B07934FEAF12383EA0A
:10661800B11383EA716A08AB53F828301A440AEBBD
:10662800020327EA010A01EA0C028AEA02021A4472
:106638004FEA743A86EA05035A4423408AEAB40AC0
:1066480006EA050B83EA0B0B8AEAB45A08F101083B
:10665800DA44B8F1400F02EB0903BB465244A9469D
:1066680019D172440265009A22444265019A324463
:106678008265029A2A44C265039A1A44049B0266F8
:106688000B444366059B63448366069B3B44C36691
:1066980049B0BDE8F08F674635468C462646194610
:1066A8001446AEE714C9060030B5E0B10F4A1049E8
:1066B80000240025C0E91245C0E914120D4C0E4A09
:1066C8000E4DC0E916420E4AC0E918520D4A8266BC
:1066D80002F17452A2F523020023A2F69242036447
:1066E800C266184630BD0E20FCE700BF85AE67BB0A
:1066F80067E6096A72F36E3C3AF54FA57F520E5170
:106708008C68059BABD9831F70B5F0B1DAB900204E
:106718001CE00C468D180026AC42F8D0036C14F827
:10672800012BC2540133402B0364F5D10146FFF716
:106738001DFFD0E9123213F5007342F10002C0E9DF
:1067480012320664E8E70029E3D10E2070BD70B567
:106758000D4616460446002876D0002974D0036CEE
:106768008022591C372BE25408443FD8C3F1370222
:10677800002105F05CFAD4E91223216C0820E1FB22
:106788000023C4E9122312BAE26323FA00F284F860
:106798003B3084F83A201A0C1B0E214684F8392025
:1067A80084F838302046FFF7E1FE691E6EB30023F7
:1067B800E26EDA4001F8012FA26EDA400A71626EC9
:1067C800DA400A72226EDA400A73E26DDA400A741D
:1067D800A26DDA400A75626DDA400A76226DDA40F7
:1067E8000833202B0A77E3D1002070BD4029C3F17C
:1067F8003F024FF0000188BF002205F018FA214639
:106808002046FFF7B3FE3822B2E71823226DDA409C
:1068180001F8012F626DDA400A71A26DDA400A723E
:10682800E26DDA400A73226EDA400A74626EDA4068
:106838000A75A26EDA400A76E26EDA40083B13F176
:10684800080F0A77E2D1CFE70E20CEE7F0B578B38C
:1068580071B36BB300241C608E18DB274FF0DC0C7F
:106868004FF0DD0E1A688E4202F1010400EB0205BA
:1068780004D11C60C0232B700020F0BD0D78C02D02
:1068880005D0DB2D0CD01C600C78845406E01C600D
:1068980087541A68541C1C6000F802C00131E1E7F3
:1068A8001C6085541A68541C1C6000F802E0F5E767
:1068B8000E20E2E710B580B3D0E902239A422ED029
:1068C8000378012B0FD0022B21D053B9C02928D02F
:1068D800DB2902D10123037003E04368541C846060
:1068E8009954112006E0DC2905D0DD290AD00223BD
:1068F80003700B2010BD511C43688160C02199545E
:106908000023E8E7511C81604368DB21F7E7C029D1
:10691800E7D1002303708360E3E70E20EAE7042051
:10692800E8E71846E6E700001FB503788DF8003061
:106938004368019383688DF80830C368054A039358
:10694800054B684653F8213052F82110984705B096
:106958005DF804FB6012002064120020F0B50646C2
:106968000F4B16F804CB43F82C200E4B17460C4659
:106978000A6943F82C200FCC89B06D460FC594E8FE
:106988000F00002F85E80F00074ACDF810C008BF98
:106998003A466946304600F069F909B0F0BD00BFD3
:1069A800641200206012002031690600024AD2F801
:1069B8000034002BFBD0704700E001400A4908B5BD
:1069C8000223C1F80435BFF36F8FBFF34F8FC1F8AF
:1069D8000805FFF7EBFF0023C1F80435BFF36F8FFD
:1069E800BFF34F8F08BD00BF00E0014010B5094C50
:1069F8000123C4F80435BFF36F8FBFF34F8F0160D5
:106A0800FFF7D4FF0023C4F80435BFF36F8FBFF33B
:106A18004F8F10BD00E0014070B50E4E01231546A2
:106A2800C6F80435BFF36F8FBFF34F8F0024AC4215
:106A380007D10023C6F80435BFF36F8FBFF34F8F1C
:106A480070BD51F8243040F82430FFF7AFFF01340F
:106A5800EDE700BF00E0014010B5054C23681BB905
:106A680004495120FFF72AF82368BDE81040184769
:106A78006812002014CA060038B50D4628B90C491A
:106A88007720FFF71BF8002038BD0A4B9842FAD14F
:106A98000020FEF7D7FF084B1C7914B901221D60AE
:106AA8001A710020FEF7DEFF002CECD01120EBE776
:106AB80014CA0600002000406812002018B90649D0
:106AC8009B20FEF7FBBF054B984201BF044B0022F9
:106AD8001A601A71704700BF14CA060000200040EF
:106AE800681200200023435082B043580193019B51
:106AF80002B070471FB501238DF80030044BCDE973
:106B08000110D3E900126846904705B05DF804FB10
:106B18007012002008B543090CBF4FF0FF33002363
:106B280000F01F0023FA00F0C30704D403494FF410
:106B3800F670FEF7C3FF4FF0A04008BD28C006005E
:106B480010B50446FFF7E6FF04F5E074022340F8A9
:106B5800243010BD7FB5434AD2F82461002E60D09E
:106B680010464FF49271FFF7BDFF02238DF80030F5
:106B7800D2F88034C2F880340393D2F83C350293BB
:106B8800394BDA6801920022C3E906226846D3E944
:106B9800001290473348D0F8443173B14FF4A271D2
:106BA800FFF7A0FF304B9A693AB10022C3E90622E9
:106BB800D968D0F83C05FFF79DFF2A48D0F8203166
:106BC800ABB14FF49071FFF78DFF0123C360264BE3
:106BD8005A6962B1D0F84C150291002299688DF873
:106BE800002001915A616846D3E9001290471D4878
:106BF800D0F858319BB14FF4AC71FFF773FF1A4BC3
:106C08005A6962B1D0F84C150291002299688DF842
:106C1800002001915A616846D3E90012904704B0F8
:106C280070BDD2F81031002BB4D04FF488711046E3
:106C3800FFF758FF0C4BD2F83C0599698842A9D157
:106C4800DC69D96864B1D2F8005225F02005C2F891
:106C580000521A699C61DA60DE61FFF74BFF99E721
:106C68009C61FAE700200040701200202DE9F047EF
:106C7800054692460C4619B97049CF20FEF71EFF0B
:106C880095F804806E4E242303FB086393F82030A4
:106C9800002B40F0CF806B492868FFF7EDFE0746D0
:106CA800002840F0C980D4F80090B9F1FF3F11D016
:106CB8004846FFF72FFF012303FA09F3D4F80090A1
:106CC800C0F808354846FFF725FF09F5E0790323A2
:106CD80040F82930D4F80490B9F1FF3F07D048466E
:106CE800FFF718FF09F5E079002340F829302B68F1
:106CF800A269C3F82425217D627D0A43C3F86C2567
:106D0800D4E900200129C3F80C25C3F814052AD1B9
:106D1800D4F80890B9F1FF3F07D04846FFF7FAFECC
:106D280009F5E079002340F82930D4F80C90B9F13E
:106D3800FF3F11D04846FFF7EDFE012303FA09F3A0
:106D4800D4F80C90C0F808354846FFF7E3FE09F57B
:106D5800E079032340F82930D4E902212B68C3F8ED
:106D68000815C3F81025242303FB08F3F218C2F80A
:106D780004A02269F250BAF1000F4AD0286894F8AA
:106D88001C90314A4FF48871FFF7ACFE28684FF425
:106D98009071FFF7A7FE28684FF49271FFF7A2FEE3
:106DA80028684FF4A271FFF79DFE28684FF4AC7174
:106DB800FFF798FE2C68B9F1070FC4F804234FEACF
:106DC800143A44F3073403D920496B20FEF776FEC2
:106DD800002CAEBF04F160431D4B0AF00F0A4FEAC6
:106DE8004919A8BF03F561435FFA89F9B4BF03F8ED
:106DF8000A9083F800932B681A0B43F30733002B90
:106E080007DB02F01F0101228A405B09114941F8A2
:106E180023202B680822C3F80025242303FB0866D7
:106E28000023C6E906337361012386F8203038460B
:106E3800BDE8F0870827FAE71127F8E799CA06009E
:106E4800701200205D6B06001003420018CB06008C
:106E580014ED00E000E100E02DE9F8433D4D06792E
:106E68000468242303FB065302465B68ABB13A4B24
:106E7800C4F8083344F30733002B4FEA14310CDB12
:106E880001F01F005B09012181402033334840F89D
:106E98002310BFF34F8FBFF36F8FD4F8003223F066
:106EA8002003C4F80032242303FB06539B6933B143
:106EB8004FF4A2712046FFF715FE012363604FF4DB
:106EC800AC712046FFF70EFE0123E360242303FB89
:106ED8000653D4F858110029FBD0996919B1D4F890
:106EE80044110029F5D00023C4F800351368D3F8FD
:106EF8000C05D3F81495D3F80875D3F810854FF01E
:106F0800FF329042C3F80C25C3F81425C3F80825AE
:106F1800C3F8102501D0FFF713FEB9F1FF3F02D0E7
:106F28004846FFF70DFEB8F1FF3F02D04046FFF795
:106F380007FE7B1C02D03846FFF702FE2046FFF70B
:106F4800BDFD242303FB0655002385F820306B6024
:106F5800BDE8F883701200201003420000E100E051
:106F68000279044B242101FB02335869003818BF09
:106F780001207047701200202DE9F047384F90F833
:106F88000490242303FB0973054693F82030012B52
:106F98008846924604D0334940F25310FEF78EFDDE
:106FA800B8F1000F04D12F494FF4AA70FEF786FDFF
:106FB800BAF1000F04D12B4940F25510FEF77EFDBF
:106FC8002B7913B9BAF1FF0F04D926494FF4AB70E6
:106FD800FEF774FD08F06043B3F1005F39D128462D
:106FE800FFF7BEFF0446002835D1242606FB0976A4
:106FF8002868C6F814A04FF49071C6F80880FFF707
:1070080071FD4FF4AC712868FFF76CFD2B6872694D
:10701800B168C3F84415C3F8482501229A6072681C
:10702800DAB9D3F82021D3F858011AB90028F8D0D2
:107038000F2007E00028FBD10122DA60D3F858219D
:10704800002AFBD0242303FB097700237B61BDE8DA
:10705800F0871020FBE71120F9E72046F7E700BF8B
:107068007012002099CA06002DE9F041474E0479B4
:10707800242303FB0463054693F82030012B88463C
:10708800174604D042494FF4D370FEF717FDB8F104
:10709800000F04D13E4940F2A710FEF70FFD27B9B3
:1070A8003B494FF4D470FEF709FD2B790BB9FF2F3C
:1070B80004D9374940F2A910FEF700FD08F06043F3
:1070C800B3F1005F5FD1242303FB0463596821B146
:1070D8002B684FF40472C3F80823242303FB0463CA
:1070E8009A6952B1DA69002A3BD021B12B684FF472
:1070F8000472C3F80423112031E09F61C3F80C80A7
:10710800DA6128684FF48871FFF7ECFC28684FF4BF
:10711800A271FFF7E7FC2B68C3F83485C3F838750C
:1071280022BB01221A602C79242202FB04625268D5
:107138001ABBD3F81011D3F84421D3F82401114312
:1071480002D10028F5D00A46242303FB0466002355
:10715800984218BF03209A42B36118BF0F20BDE8B8
:10716800F081C3F81080DF610122CAE7D3F800225A
:1071780042F02002C3F80022D5E74FF40472C3F8A6
:1071880004230020EBE71020E9E700BF701200207D
:1071980099CA060028B139B10023C1E90030184660
:1071A800704748F21050704748F21350704730B19A
:1071B800036848F240508B4208BF0020704748F2ED
:1071C8001050704728B148F21150914208BF002072
:1071D800704748F21050704770B506460C461D4679
:1071E800FFF7D8FF50B9B3794AB1AB420AD111467B
:1071F8002046FDF774FE08B9044B236070BD48F2C1
:107208001050FBE748F21150F8E700BF7052464DA6
:107218002DE9F0470C4606460F492046DDE9088966
:1072280015461F46FFF7C3FFA0B963685A79494658
:1072380052004046FFF7C6FF60B94DB1CDF8208037
:107248003B462A4621463046BDE8F047FDF74FBE8B
:1072580048F21050BDE8F0877052464D10B504460C
:1072680038B149B10B684160984708B9044B2360AD
:1072780010BD48F20150FBE748F21050F8E700BF94
:107288006E524648F0B4134648B10768094EB742F3
:107298000AD161B12AB14368F0BC5B68184748F26B
:1072A80001531846F0BC704748F20253F9E748F218
:1072B8001053F6E76E524648F0B460B107680C4EBA
:1072C800B7420CD171B143681568DC68A5420CD38C
:1072D800F0BC9B68184748F20150F0BC704748F270
:1072E8000250FAE748F21350F7E748F21450F4E76F
:1072F8006E524648F7B50446DDE90867154601931E
:10730800FFF7ACFF68B9019A29462046FFF7BAFF94
:1073180038B93A463146204603B0BDE8F040FFF799
:10732800CBBF03B0F0BD0000F8B50A4F0A4C0B4EB6
:10733800E41B0123E40833700025A54203D102238E
:1073480033700020F8BD57F8353098470028F9D138
:107358000135F2E740BD060040BD0600941200204A
:1073680038B50D46044618B908493320FEF7A6FB80
:10737800691E21442046814200D238BD03780A782C
:1073880000F8012B01F80139F5E700BF4ACB0600E8
:1073980070B50D461446064618B90A494520FEF749
:1073A8008DFB1DB907494620FEF788FB621E324453
:1073B800013DB24200D270BD15F8013F02F8013913
:1073C800F7E700BF4ACB060070B5164604460D46DF
:1073D800FFF7DEFF3246A919A019BDE87040FFF794
:1073E800D7BF38B50D460446FFF7BAFF29466019DE
:1073F800BDE83840FFF7B4BF08B507281BD8DFE859
:1074080000F004121A1A1A041A040120FDF731FDBB
:107418000020FDF7F3FC0120FDF7F0FCBDE8084073
:107428000220FDF701BD0120FDF7FEFCBDE8084084
:107438000220FDF7E3BC08BD08B5FDF791FBFDF799
:1074480073F90028FBD10D4D642445F001054FF474
:107458007A40A847013CFAD1094BD3F8F020D2076B
:1074680000D500BEBFF34F8FD968064A01F4E0612A
:107478000A43DA60BFF34F8F00BFFDE7A0CC0600D8
:1074880000ED00E00400FA0507B50B46064C074975
:107498000092641AE40824040246054944F00100F5
:1074A800FDF7B9FAFFF7C8FF58BD060048BD06004A
:1074B80014CC060008B50246054B064806491B1AB7
:1074C800DB081B0443F00100FDF792FAFFF7B4FF55
:1074D80058BD060048BD06004BCC060010B501F0AB
:1074E80037FE4FF48051002001F00DFA08B1FFF784
:1074F800E1FF1548C0F5FC2101F005FA0146002816
:10750800F5D11248124CFDF7BFF8FCF7EDFF114B0F
:107518001149E41AE408240444F00300FDF764FA6E
:107528000E4801F09DF80028E1D1FDF7FDF800288C
:10753800FBD10B4944F00100FDF756FAFDF7F4F8CA
:107548000028FBD1D3E700BF00400600918C06005D
:1075580058BD060048BD060066CC0600017406004A
:1075680072CC06008B1810448B4200D1704713F878
:10757800012D00F8012DF7E7C3F10803DB0070B512
:1075880001330446002003A55B1920C940CAAD1980
:1075980020C4184720C940CA754120C420C940CA20
:1075A800754120C420C940CA754120C420C940CAB9
:1075B800754120C420C940CA754120C420C940CAA9
:1075C800754120C420C940CA754120C4404170BDDE
:1075D8000000000000000000C3F10803DB0070B5E4
:1075E8000133002403A500BF5B1920C940CAAD1BA5
:1075F80020C0184720C940CAB54120C020C940CA88
:10760800B54120C020C940CAB54120C020C940CAE0
:10761800B54120C020C940CAB54120C020C940CAD0
:10762800B54120C020C940CAB54120C06441B4FA60
:1076380084F0400970BD00BF2DE9F04F08B4F8CAC6
:1076480004B451F8042BA3FB028940F8048B4FF0D3
:10765800000AE4FB629A4FF0000BE5FB62AB4FF0C7
:10766800000CE6FB62BC4FF0000EE7FB62CE51F85F
:10767800042B4FF00008E3FB628940F8048BE4FB1D
:10768800629AE5FB62ABE6FB62BCE7FB62CE51F8AF
:10769800042B4FF00008E3FB628940F8048BE4FBFD
:1076A800629AE5FB62ABE6FB62BCE7FB62CE51F88F
:1076B800042B4FF00008E3FB628940F8048BE4FBDD
:1076C800629AE5FB62ABE6FB62BCE7FB62CE51F86F
:1076D800042B4FF00008E3FB628940F8048BE4FBBD
:1076E800629AE5FB62ABE6FB62BCE7FB62CE40F860
:1076F800049B40F804AB40F804BB40F804CB40F8C6
:1077080004EB0CBC052B00F01E810C68A0F11400E2
:10771800A1F11401A2F1140252F804EB4FF0000594
:1077280050F8046BE4FB6E5652F804EB50F8047BF7
:10773800E4FB6E6752F804EB50F8048BE4FB6E78B8
:1077480052F804EB50F8049BE4FB6E8952F804EB02
:1077580050F804ABE4FB6E9AA0F1140052F8044B05
:1077680051F804EB4FF0000CE4FB6EC540F804CB75
:1077780051F804EBE4FB6E5640F8045B51F804EB57
:10778800E4FB6E6740F8046B51F804EBE4FB6E7899
:1077980040F8047B51F804EBE4FB6E8940F8048B55
:1077A80051F804EBE4FB6E9AA0E80006062B00F003
:1077B800CA800C68A0F11800A1F11801A2F1180202
:1077C80052F804EB4FF0000550F8046BE4FB6E56DA
:1077D80052F804EB50F8047BE4FB6E6752F804EBB4
:1077E80050F8048BE4FB6E7852F804EB50F8049BD5
:1077F800E4FB6E8952F804EB50F804ABE4FB6E9A94
:1078080052F804EB50F804BBE4FB6EABA0F118008F
:1078180052F8044B51F804EB4FF0000CE4FB6EC532
:1078280040F804CB51F804EBE4FB6E5640F8045BD7
:1078380051F804EBE4FB6E6740F8046B51F804EB75
:10784800E4FB6E7840F8047B51F804EBE4FB6E89A6
:1078580040F8048B51F804EBE4FB6E9A40F8049B63
:1078680051F804EBE4FB6EABA0E8000C072B6AD0E0
:1078780008B40C68A0F11C00A1F11C01A2F11C02C3
:1078880052F804EB4FF0000550F8046BE4FB6E5619
:1078980052F804EB50F8047BE4FB6E6752F804EBF3
:1078A80050F8048BE4FB6E7852F804EB50F8049B14
:1078B800E4FB6E8952F804EB50F804ABE4FB6E9AD3
:1078C80052F804EB50F804BBE4FB6EAB52F804EB3F
:1078D80050F804CBE4FB6EBCA0F11C0052F8044B3A
:1078E80051F804EB4FF00003E4FB6E3540F8043B1D
:1078F80051F804EBE4FB6E5640F8045B51F804EBD6
:10790800E4FB6E6740F8046B51F804EBE4FB6E7817
:1079180040F8047B51F804EBE4FB6E8940F8048BD3
:1079280051F804EBE4FB6E9A40F8049B51F804EB21
:10793800E4FB6EAB40F804AB51F804EBE4FB6EBC1F
:10794800A0E8001808BCBDE8F08F002310B51C465D
:107958005AB2914200DC10BD40F823400133F7E7EA
:1079680010B500231A465CB2A14203DCB2FA82F0D9
:10797800400910BD50F8234001332243F3E74A1170
:10798800012350F8220001F01F0103FA01F1084019
:107998007047013910B549B2041D0A06CBB204D4A8
:1079A800013954F82120002AF7D001335BB273B1B2
:1079B80003F18042013A50F82220002022B9013B0D
:1079C80000EB431318B210BD52080130F6E7184611
:1079D800F9E710B500235CB2A24200DC10BD51F8F3
:1079E800234040F823400133F5E710B5013A52B27D
:1079F800130601D5002010BD50F8224051F822305E
:107A08009C4205D802F1FF32F2D24FF0FF30F2E784
:107A18000120F0E700EB81010023884200D3704782
:107A280051F8042D43EA52030B60D307F5E737B545
:107A38001D469DF9183001930446FFF79DFD019BF3
:107A480038B91A4621462846FFF7CFFF0128019B7F
:107A580007D02A462146204603B0BDE83040FFF74C
:107A6800BBBD03B030BD37B51D469DF91830019335
:107A78000446FFF7B1FD019B38B12A46214620464E
:107A880003B0BDE83040FFF777BD03B030BD2DE946
:107A9800F04FB5B004AC9DF9F8501F4680462B4610
:107AA8002046FFF7C9FD24AB29463846CDE9023404
:107AB800FFF76FFFC0EB851004B2002C2146B8BF5A
:107AC80004F11F01634203F01F0341F3471104F05F
:107AD8001F0614A858BF5E42FFF737FF002E08B2F2
:107AE8002BDD14AB002203EB8000C6F1200E1346F9
:107AF800AB4217D36B00019314AB03EB85096F1EE0
:107B080034AB012603EB8707002C54DA34AB03EBC4
:107B180086062A4656F8C81C4046FFF75AFF35B075
:107B2800BDE8F08F57F823C00CFA06F10A4340F875
:107B3800042B01332CFA0EF2DAE714AB2A46394645
:107B480003EB8000FFF745FFD4E70FFA82FE5AF8EF
:107B5800C83C53F82EB034AB03EB8202013052F824
:107B6800803C0B44BBEB030334BF012200229B453E
:107B780018BF11465CF8C82C42F82E30019B42B25F
:107B88009A42E2DB731A5E42294614A85E41FFF767
:107B980041FF34AB03EB8503294653F8802C57F893
:107BA800803C43EAC27347F8803C4846013CFFF7F3
:107BB80031FF24B2A8E734AB0020C6F1010C01461E
:107BC80003EB860A03EB8C0CD8E730B51C4691B062
:107BD800054693F900306846FFF72EFDD4F8AC301F
:107BE80069462846984711B030BD13460A46FFF744
:107BF800ECBF2DE9F04793F9006092B0044689463E
:107C08001046314615461F46FFF7AAFE002840F0E9
:107C180091803A46494602A8FFF7E7FF3B4602AA89
:107C280021460AA8FFF7D1FF02A908463A46FFF7FE
:107C3800DCFF3B462A4649464846FFF7C6FF07F1A0
:107C480004083A4629462846FFF7CFFF43462A4606
:107C5800214620460096FFF7EAFE43462A46294673
:107C680028460096FFF7E3FE43462A462146284663
:107C78000096FFF7F8FE3B462A4621462046FFF7C6
:107C8800A4FF43462246214628460096FFF7CFFE2A
:107C9800434600962A4621462046FFF7C8FE236839
:107CA800DB074AD53346424621462046FFF764FCA7
:107CB800314682462046FFF7ADFE06F18043013B80
:107CC80054F8232042EACA7244F823203A4621464F
:107CD8002846FFF78AFF43460AAA294628460096FF
:107CE800FFF7C1FE43460AAA294628460096FFF731
:107CF800BAFE0AA9084643462A460096FFF7B3FE8D
:107D08003B460AAA21462046FFF75FFF02AA4346E0
:107D1800104621460096FFF7A6FE32462946204621
:107D2800FFF757FE49462846FFF753FE02A9484683
:107D3800FFF74FFE12B0BDE8F08731462046FFF747
:107D480069FEC3E72DE9F04115468AB004460E46A0
:107D58001C22002103A803F06AFF2F1D95F900805B
:107D680003232A46314620460293FFF73EFF3B464F
:107D780002AA21462046CDF80080FFF774FE2B4664
:107D8800324621462046FFF720FFCDF800803B46CB
:107D980005F1840221462046FFF749FE0AB0BDE8F6
:107DA800F08100002DE9F042082288B0FFF711FEAB
:107DB800CB6A03930B6B04934B6B05938B6B069306
:107DC800CB6B07930C4681460027134669466A46E3
:107DD8006846CDE901770097FFF7CEFB08230546F3
:107DE8006A4649464846FFF7C7FB236B0393636B14
:107DF8000493A36B0593E36B0544CDE906376A4604
:107E0800082369466846FFF7B7FB082305446A4616
:107E180049464846FFF7B0FB236A0093636A01931B
:107E2800A36A0293A36B0693E36B079305440823A5
:107E38006A4649464846CDE904770397FFF79CFB15
:107E4800636A0093A36AA26B0193E36A02930492A4
:107E5800636BE26B0393CDE90523236A07932E181E
:107E680008236A4649464846FFF786FBE36A0093BB
:107E7800236B0193636B0293236A0693A36A0793A8
:107E8800351808236A4649464846CDE904770397DA
:107E9800FFF7A2FB236B0093636B0193A36B029321
:107EA800E36B0393636A0693E36A07932E1A082326
:107EB8006A4649464846CDE90477FFF78DFB636B70
:107EC8000093A36B0193E36B0293236A0393636AA2
:107ED8000493A36ACDE90537236B0793361A082361
:107EE8006A4649464846FFF777FBA36B0093E36B66
:107EF800CDE90137636A0393A36A0493E36ACDE982
:107F08000537636B0793361A08236A46494648467D
:107F1800FFF762FB361A0E4C0FD436B908224946D1
:107F28002046FFF762FD01280FD008232246494664
:107F38004846FFF751FB361AEFE708232246494621
:107F48004846FFF719FB3618F7D408B0BDE8F082A9
:107F5800ACCC060070B514468AB006460D461A46E3
:107F6800214602A80193FFF740FE019B02AA314671
:107F78003046FFF72AFE02A9019B22460846FFF772
:107F880024FE019B02AA29462846FFF71EFE0AB0D6
:107F980070BD2DE9F0478AB01446DDF848A0554673
:107FA8001F4615F9046B0096804689462B46024603
:107FB800214602A8FFF757FD02A952460846FFF7D7
:107FC80014FE534602AA41464046FFF7FEFD5346BB
:107FD80002AA21462046FFF7F8FD2B464A463946B5
:107FE80038460096FFF73FFD5246394602A8FFF78C
:107FF800FCFD02A92B46424608460096FFF733FDD2
:1080080002A92B46224608460096FFF72CFD2B4670
:108018004246214620460096FFF725FD5346224654
:1080280049464846FFF7D1FD2B4602AA414620465D
:108038000096FFF718FD5346224639463846FFF7A3
:10804800C4FD2B464A46394638460096FFF70BFDD5
:10805800324602A92046FFF7BCFC0AB0BDE8F0870B
:108068002DE9F0471F46B3F9023013F11F0448BF4A
:1080780003F13E04DD1D48BF03F10E056611EC1047
:10808800944275B228BF144689462946FFF75DFC1D
:10809800224649468046FFF765FAB7F90230B3EB46
:1080A800C40F4FEAC4021FD2D21A08EB860400217B
:1080B800C2F12006A0450ED324372A464146384649
:1080C800FFF793FC01280FD02B463A464046BDE8FF
:1080D800F047FFF781BA54F8040D20FA02F30B4376
:1080E800236000FA06F1E5E7BDE8F08770B503689C
:1080F80013F001060546144605D013460A46014604
:10810800FFF73AFA064621462846FFF783FC46B1B0
:1081180004F18042013A55F8223043F0004345F813
:10812800223070BDF0B50F46A1B006461946384654
:1081380015461C46FFF714FC28B1304621B0BDE8AF
:10814800F040FFF702BC224639466846FFF741FC7B
:10815800294608A8FFF73DFC10A82146FFF7F5FBC4
:10816800012318A81093FFF7F0FB224608A96846D8
:10817800FFF73BFC30B9224610A93046FFF729FC2F
:1081880021B0F0BD009BDA0709D421466846FFF705
:1081980041FC2246294610A8FFF7A8FFE5E7089BFF
:1081A800DB0707D4214608A8FFF734FC22462946F6
:1081B80018A8F1E7002823461CDD08AA6946684686
:1081C800FFF70AFA21466846FFF724FC224618A959
:1081D80010A8FFF70AFC002805DA10A923462A464A
:1081E8000846FFF7C9F910A9234618AA0846FFF759
:1081F800F3F9CEE76A4608A8FFF7EEF9214608A882
:10820800FFF708FC224610A918A8FFF7EEFB002884
:1082180005DA18A923462A460846FFF7ADF918A932
:10822800234610AA0846FFF7D7F9BFE7004870476A
:10823800A8CC06002DE9F04F2DED028BEBB00D46D2
:10824800769E03901946B6F9023096F9004013F16C
:108258001F0848BF03F13E0848F3471808F1FF3BE1
:1082680022AB002743F82B706AAB03EB8B034AA8B9
:1082780043F8807C43F8607C924696F90120FFF72A
:1082880071F996F9012052A81144FFF76BF92146BC
:108298004AA8FFF765FB8146002840F0278152A8CD
:1082A800FFF75EFB0290002840F0228106F12409C6
:1082B80042464AA94846FFF798FB012840F01A8130
:1082C800424652A94846FFF790FB0128049040F027
:1082D80011810AAF43464A461AA8FFF723FF029BBB
:1082E80047F82B305246294638463346FFF7B8FE42
:1082F800394638464B461AAACDF80080FFF7C7FB27
:108308005AAD4B461AAA4AA912A8CDF80080FFF721
:10831800BEFB224628460399FFF75BFBA3000593A3
:10832800039B05EB840A03EB840106F1440B5046DA
:10833800FFF74FFB594632A8FFF74BFBA3000BEBA7
:1083480003013AA8FFF745FB331D294632AA1AA8AC
:10835800009408EE103AFFF786FB53462A463AA9DE
:1083680032A80096FFF715FE1AA9084618EE102A3B
:108378002346FFF7D7FE1AAA514628463346FFF789
:10838800E9FD029BCDE9063B039B41463846CDE912
:108398000835FFF7FEFA4146834612A8FFF7F9FAB7
:1083A8005845B8BF584685B2691E09B23846039188
:1083B800FFF7E5FA0399071E12A818BF0127FFF770
:1083C800DEFA002814BF022000200DF1180A074326
:1083D80022465AF8271022A8FFF7FBFA0DF1A80B3E
:1083E800A30019445846FFF7F4FA1AA82146FFF7E4
:1083F800ACFA049B0360023D22AB2DB20393824684
:10840800002D26DA18EE102A234651465046FFF76B
:1084180089FE0398334652465946FFF79BFD039958
:1084280042464846FFF7E1FA012804D043464A4647
:108438000846FFF7D1F8013C64B24AAA23064AD598
:10844800029BB3FA83F040096BB0BDEC028BBDE828
:10845800F08F33465246D6F8A47003985946B84769
:1084680029460AA8FFF78BFA2946071E12A818BF43
:108478000127FFF784FA002814BF022000200743D1
:1084880006AB53F8271019B3224632A8FFF7A1FA12
:10849800059B3AA81944FFF79CFA01463346524611
:1084A80032A8FFF757FD18EE103A0399009432AA44
:1084B80042A8FFF7D8FA039A00965B463AA932A871
:1084C800FFF767FD334642AA51465046FFF77DFB4A
:1084D800013D2DB294E7039B52F8241053F8243041
:1084E8004B40029919430291013CA7E73846ABE794
:1084F8004846A9E70298A7E713681F2B10B514464A
:1085080007D900220830FEF722F908B92023236092
:1085180010BD48F21450FBE70830FEF7F5B80830F4
:10852800FEF7C2B8014B01221A707047B816002036
:1085380008B5FCF715FBFCF7F7F80028FBD1BFF3EB
:108548004F8F0549054BCA6802F4E0621343CB60BC
:10855800BFF34F8F00BFFDE700ED00E00400FA0510
:1085680008B50948094B0A49C01AC008000440F078
:108578000400FCF739FA074B074800221A70BDE8D7
:10858800084001F043BF00BF58BD060048BD0600C3
:1085980070CD0600B81600203985060008B50748D2
:1085A800074B0849C01AC008000440F00300FCF754
:1085B8001BFABDE80840FFF7D3BF00BF58BD06004F
:1085C80048BD060086CD0600042810B5044609D823
:1085D80002280DD812D00B4B1B6893B12046BDE87A
:1085E80010401847831F012BF5D8FFF7B9FFF2E7B2
:1085F80005494FF4341000F007FBECE701F0F0FDFB
:10860800E9E710BDBC160020A585060008B543099A
:108618000CBF4FF0FF33002300F01F0023FA00F0D7
:10862800C30704D403494FF4F670FDF747FA4FF037
:10863800A04008BD28C0060008B50648064B0749F3
:10864800C01AC008000440F00400FCF7CDF900206F
:1086580008BD00BF58BD060048BD06009ACD0600FB
:10866800F8B5724B724C7349E41AE408240444F0D8
:10867800040605463046FCF7B7F96F4B10201D601D
:10868800FFF7C4FF6D4BC0F84037002001F0D4FE5F
:10869800002840F0C68000F065FC012800F0BA8090
:1086A800022800F0C080002840F0BB804FF08043D3
:1086B800D3F8005415F480354CD04FF48032C3F809
:1086C800002405465E4F3B6A012B56D05D4944F0B5
:1086D8000300FCF789F95C493046FCF785F94FF44B
:1086E800341400F093FD594A20211820FDF7DCF8D6
:1086F80008B1FEF7DFFE4FF08043D3F81C2502F0E7
:10870800F802B02A09D1D3F81C25D20742BFD3F802
:108718001C2502F04E02C3F81C25FFF78DFF002828
:108728007FD120464A4900F06FFA4A4800F032FFEC
:10873800002876D148493046FCF756F900F0ACFDE0
:10874800FDF732F9FBF7F0FF0028F7D120BF40BF53
:1087580020BFF3E7D3F8202502F0F802A82A0AD1AF
:10876800D3F82025D00706D5D3F8202502F05602E5
:10877800C3F82025A6E70125A4E74FF440535A681B
:10878800364B9A420FD17A6B1DB997F86032012B9C
:1087980009D033484FF4805102F0A4FC18B931498C
:1087A80044F0020095E701F051FFBA6901461DB98E
:1087B80097F8A132012B05D02B4802F093FC08B999
:1087C8002A49EDE72A493046FCF70EF91020FFF751
:1087D8001DFFD0F81035D90301D426497CE74FF0A6
:1087E8008043D3F81C3513F0B10F01D0224973E749
:1087F80001F050FEA8B9214D2870214801F006FE6D
:108808002B7823B91F4940F21E20FDF757F900F0D5
:108818003DF801E0FFF7A4FE1B4944F00100FCF716
:10882800E3F80320F8BD4FF4A0245AE748BD06003A
:1088380058BD0600B4CD0600BC1600200C0003008D
:10884800DC1F0020CBCD060069CE06009812002060
:10885800A5850600D1850600D8CE0600DBE5B15116
:108868003C220020F9CD06007D22002034CE0600EF
:108878005CCE06008CCE0600ABCE0600B8160020F3
:108888002D850600E8CE0600CCCE060037B5164B7F
:10889800164C174D1749E41AE408240444F0040060
:1088A8004FF480520190FCF7A3F8D5F880201249C4
:1088B8000198FCF79DF84FF0FF33C5F88030C5F8F4
:1088C800803100F08AFF20B10C4944F00100FCF728
:1088D8008BF8FBF729FF0028FBD14FF4805003B039
:1088E800BDE8304000F03CB848BD060058BD060061
:1088F80000E100E072CF0600A8CF0600D2CF060044
:1089080080F30888084770B5C1F30B0434BBB0F591
:10891800FE2F23D84B1E1B0B020B03EB1031012635
:108928004FF08040914201D2204670BD02F01F03F3
:10893800550906FA03F3032D05D8DFE805F002060A
:10894800090CC0F800360132ECE7C0F80436FAE743
:10895800C0F81036F7E7C0F81436F4E70724E3E761
:1089680038B504462648C0F50021FFF7CCFF054678
:1089780068B12448244B25491B1ADB081B0443F023
:1089880001002A46FCF734F82846FEF793FD01F06B
:108998005DFE1F4B9B6903F6FF7323F47F6323F08F
:1089A8000F0319180020FFF7AEFF054668B11548F8
:1089B800154B18491B1ADB081B0443F001002A4613
:1089C800FCF716F82846FEF775FDEFF3058200233D
:1089D800D4E9005483F3148883F3108883F311884F
:1089E80083F31388C2F308021AB10B495820FDF724
:1089F80065F821462846BDE83840FFF781BF00BF2B
:108A08000040060048BD060058BD060007D0060015
:108A1800DC1F00203ED0060072D0060073B5274B3D
:108A2800064627481B1ADB081B040C463246254914
:108A380043F00400FBF7DCFFB4F1807F39D322490F
:108A48008F20FDF73BF86FF07F41A14228BF2146F8
:108A58001E4B641AD3F80455631E942B96BF9634A4
:108A6800746074600D44347B25F07F4598BF963D53
:108A7800032C03D914497720FDF720F8134E04F589
:108A8800A8734FF4F86046F82350114B43F00103E4
:108A98009847104BA200134400221A601B680193E8
:108AA800019B4FF4803303FA04F4C6F8044302B080
:108AB80070BD952CC7D804499020C2E758BD060060
:108AC80048BD06000CD1060022D106000040024035
:108AD800E0D10600404102401FB518490B7853BB4E
:108AE8004FF08043A024D3F81824D2035CBF01229E
:108AF8009A60134B0022C3F80021D3F800010390B9
:108B08000398C3F84021D3F8400102900298C3F8B3
:108B18004421D3F84401019001980A4880F824437D
:108B2800102444600220C3F8082501229A601A60C4
:108B3800C3F804030A7004B010BD00BFC4160020B7
:108B48000040024000E100E0264B2DE9F743D3F84E
:108B5800042152B124490A6801320A600022C3F88C
:108B68000421D3F804310093009B204D204B214C65
:108B7800214EDFF89080DFF86C90204FED1AED0859
:108B88002D0445F004053368CBB100233360336806
:108B98000193224641462846019BFBF729FF227B89
:108BA80017494FF480339340C9F8083322462846C2
:108BB800FBF71EFF616851B12046FFF72FFF04360F
:108BC800BE4204F11004DED103B0BDE8F083A16811
:108BD80011B12046FFF722FF2368002BEFD09847FA
:108BE800EDE700BF00400240C016002058BD060057
:108BF80048BD060024000020404102404841024090
:108C0800C9D10600B7D10600F8B5114B114E04467C
:108C1800114837681B1ADB081B043A4643F0040066
:108C28000D460E49FBF7E4FE3A7B4FF48033934040
:108C38000B4AC2F808334CB13668FFF74DFF356070
:108C480021463046BDE8F840FFF7E8BEF8BD00BF52
:108C580058BD06004400002048BD0600B7D10600F4
:108C68000040024070B5074B1D6804460E46A860D8
:108C7800FFF732FF2E6021462846BDE87040FFF717
:108C8800CDBE00BF48000020034A044B1068D3F84B
:108C9800043503EB00607047C01600200040024016
:108CA800014B01221A707047C5160020224BDA6A60
:108CB800AC2A2DE9F3415F6A9D6C1FD15B6B1D44A3
:108CC800FF1A1E4B1E4E1F4A1F490097F61AF60838
:108CD800360446F004082B464046FBF79CFE19482C
:108CE8003A46294602F043FF044668B91749404608
:108CF800FBF77AFE204602B0BDE8F081002DE0D1F6
:108D080001F0B8FC0546DCE711493B462A464046D7
:108D1800FBF777FEFBF708FD0028FBD100F0BCFA53
:108D28003946284600F048FD04460028E2D00949A3
:108D380046F00100DCE700BFDC1F002048BD06004C
:108D480058BD060000400600E6D106001BD206000A
:108D580052D206007FD206002DE9F04F3C4B164652
:108D68003C4A9B1A87B0DB081B04814205460F4624
:108D7800049343F0040B08D137495846FBF734FEF7
:108D88000024204607B0BDE8F08F03D233494F20B6
:108D9800FCF794FE36B1C5F30B031BB12F495320E2
:108DA800FCF78CFE7B1BB3F5805F4FEA133403D2CC
:108DB8002A495720FCF782FE00F028FA082C28BF21
:108DC800082406F6FF7923034FEA1939039405931B
:108DD8000EB93446D5E7039B4B453ABFDDF80CA0E6
:108DE800DDF81480CA464FF000025146284628BFD5
:108DF800B04600F09BFC04460028C2D11849CDF8C3
:108E080000802B463A465846FBF705FE08F1030258
:108E1800234622F003023946284600F049FC04465E
:108E28000028AED10F4A136B4344136301F0F4FAE0
:108E3800A9EB0A09A6EB080645444744044600285E
:108E4800C6D0049B084943F00100FBF7CDFD98E725
:108E580058BD060048BD060099D20600A8D20600F3
:108E680040D30600DC1F002061D306002DE9F7433C
:108E780001F012FC314C324BDFF8E4903149D9F85B
:108E88004860D9F83080D9F83450E41AE40824044A
:108E9800074644F004000190FBF7A6FD06F50053D1
:108EA80001985A68284B9A4209D0284944F0010091
:108EB800FBF79AFD0325284603B0BDE8F083D9F8EF
:108EC8003030AB421E4404D12149FBF78DFD00250B
:108ED800F1E7C3B94FF440521178142982BF1D49F4
:108EE8005269B2FBF1F206F5005198BF1A4691F8A3
:108EF80000C0BCF1140F82BF4969164BB1FBF3F3F4
:108F08001549FBF77EFDA5EB080202F6FF7222F475
:108F18007F6222F00F02314607EB0800FFF71CFFC3
:108F2800054628B10D4944F00100FBF75DFDC2E795
:108F380003B0BDE8F04301F06FBA00BF58BD0600AA
:108F480048BD06009AD30600DBE5B151BFD3060041
:108F5800F3D3060040420F0005D406002ED40600C5
:108F6800DC1F00202DE9F047624B634D634E6449D6
:108F7800ED1AED082D0445F004073846FBF734FDDB
:108F8800F36AAA2B00F09A800CD8012B22D0A52BCB
:108F980000F0888045F003005A49FBF725FD0020C2
:108FA800BDE8F087AC2BF5D157493846FBF71CFDD7
:108FB80056493846FBF718FDFFF758FF04460028C6
:108FC80000F08680524945F00100FBF70DFD4FF097
:108FD800010823E04F493846FBF706FDD6F82490F0
:108FE800D6F848A001F032FB346B4B4900EB04087B
:108FF8003846FBF7F9FC316B5144884514BFA9EB9F
:10900800040200224046FFF7A7FE044670B1434918
:1090180045F00100FBF7E8FC4FF00008F36A40490F
:10902800224645F00100FBF7ECFC13E001F00EFBD3
:1090380022464946FCF726FDB26A904280462AD16C
:1090480038493846FBF7D0FC0123C6E90783C6F840
:109058001890A0463448DFF8F49001F0B7FA0023DE
:10906800324889F8003001F0D7F999F80030044601
:1090780023B92F4940F2A510FCF720FD8CBBB8F1AD
:10908800000F35D0336A012B32D138462949FBF716
:10909800ABFC022084E70346274945F00100FBF7B3
:1090A800B0FCD6E725493846FBF79EFCFFF7DEFE05
:1090B8004FF001080446002CCCD0AFE720493846D1
:1090C800FBF792FCFFF7F2FD4FF000080446F2E7C9
:1090D800FFF7ECFD044608B11A4974E74FF00108A0
:1090E800B8E745F001001849FBF77EFC032057E775
:1090F800012055E748BD060058BD0600DC1F0020CA
:1091080047D4060053D50600FCD406000AD506004D
:1091180027D5060068D4060072D406002ED40600AF
:109128006CD506008DD4060000200020A98C06000E
:10913800A8D206009ED50600A2D40600EAD40600EE
:10914800F3D406003DD50600FAD50600C516002062
:1091580010B50024D4F8F83F013304D1084940F68B
:10916800F870FDF743FCD4F8FC3F013307D1BDE8A4
:1091780010404FF4FC2140F6FC70FDF737BC10BDE1
:10918800004006000A4AD2F800347BB1094800239F
:10919800D2F80815D940C90748BF03F5C07103F1D3
:1091A800010348BF42F82100072BF1D1704700BFE7
:1091B800000001403546526E08B50748074B08497C
:1091C800C01AC008000440F00300FBF70DFCBDE81E
:1091D8000840FFF7D7BF00BF68BD060048BD0600BE
:1091E80014D6060007B5084B0022C3F80021D3F8AF
:1091F80000310193019BFBF7B3FCFBF795FA0028BC
:10920800FBD103B05DF804FB0000014037B5194DF0
:109218002B784BBB18481949194B401AC008D3F88A
:109228000024000440F0030002B3D3F804451549B4
:1092380001902246FBF7DCFB40F616529442B8BF79
:109248001446A4F54864FFF79DFF01980E4922468D
:10925800FBF7CEFB0D492046FFF704FD0C4B4FF4FE
:1092680080321A6001232B7003B030BD0949FBF727
:10927800BBFBF7E7C616002068BD060048BD060020
:109288000000014022D606003BD60600C191060028
:1092980000E100E06DD60600034BD3F800340BB1B3
:1092A800FFF770BF704700BF000001404FF08053C8
:1092B800D3F83001421C04BF4FF0704393F8E00F1D
:1092C800831F5842584170474FF0704393F8E02F7E
:1092D800062A09D1D3F8E83FC3F30313033B032B52
:1092E80002D8024AD05C7047002070479BD606001F
:1092F80008B5FFF7DBFF40B14FF080538F4AD3F832
:109308002433C3F30423C2F84035FFF7DDFF10B15F
:109318008B4B8C4A5A67FFF7C9FF48B14FF080530F
:109328004FF08042D3F84432C3F34233C2F83C359D
:10933800FFF7CAFF30B1844AD2F8FC3023F08073BB
:10934800C2F8FC30FFF7B2FF40B14FF08043002273
:10935800C3F80C21C3F81021C3F83825FFF7B4FF70
:1093680020B14FF080430322C3F8A025FFF7ACFFDC
:1093780060B1764B0522C3F810260122C3F888266F
:109388000022C3F818263F22C3F814264FF0805352
:10939800D3F83021511C09BF4FF07043D3F8343152
:1093A80093F8E02FD3F8E83F08BFC3F30313062A66
:1093B8004DD1033B032B03D8654AD35C002B46D021
:1093C8004FF08052634BD2F80414C3F82015D2F83A
:1093D8000814C3F82415D2F80C14C3F82815D2F8C9
:1093E8001014C3F82C15D2F81414C3F83015D2F899
:1093F8001814C3F83415D2F81C14C3F84015D2F861
:109408002014C3F84415D2F82414C3F84815D2F828
:109418002814C3F84C15D2F82C14C3F85015D2F8F8
:109428003014C3F85415D2F83414C3F86015D2F8C0
:109438003814C3F86415D2F83C14C3F86815D2F888
:109448004014C3F86C15D2F84424C3F87025FFF70C
:109458002DFF48B14FF080534FF08042D3F8583277
:1094680003F04F03C2F8E43EFFF720FF48B14FF086
:109478008043D3F80024D20744BF6FF00102C3F839
:1094880000244FF08053D3F83021062A0ED1D3F8A8
:109498003431033B032B02D82F4AD35C33B12F4A14
:1094A800D2F83C3743F48063C2F83C37264AD2F8F6
:1094B800883043F47003C2F88830BFF34F8FBFF38E
:1094C8006F8F4FF01023D3F80022002A03DBD3F864
:1094D8000432002B2EDA224B0122C3F80425D3F8DC
:1094E8000024002AFBD04FF010221521C2F80012E8
:1094F800D3F80024002AFBD04FF010231522C3F81C
:109508000422174BD3F80024002AFBD00022C3F80A
:109518000425D3F80024002AFBD0BFF34F8F0A4953
:10952800104BCA6802F4E0621343CB60BFF34F8F5D
:1095380000BFFDE70C4B0D4A1A6008BD0030014022
:1095480000C007400DF0ADBA00ED00E0005000404B
:1095580093D6060000C0004097D6060000100040D1
:1095680000E001400400FA054C0000200090D00300
:10957800831F012B10B5044602D8002000F0ECFF31
:10958800034B1B681BB12046BDE81040184710BDAF
:10959800C816002038B5104B104C1860104B1149F4
:1095A800E41AE408240444F00300FBF71DFA002041
:1095B800FFF7DEFF0C4800F095FF054620B9BDE82F
:1095C8003840094800F06CBC0246084944F00100E4
:1095D800FBF70EFA284638BDC816002058BD06000D
:1095E80048BD060054D806007995060067D80600DD
:1095F80030B51A490B6885B004460BB1013B0B60C6
:109608001748184A63682578121AD208120442F0DB
:1096180004008BB90B68144A14490093012D08BF44
:109628000A46A3681249FBF7F6F963699BB1E0683B
:1096380005B0BDE8304018470A68029222690192D5
:10964800A2680A490092084A012D08BF0A4609493A
:10965800FBF7FBF9E9E705B030BD00BFCC160020E9
:1096680048BD060070BD060097D8060091D80600D0
:109678009DD80600C3D8060008B50848084B094914
:10968800C01AC008000440F00400FBF7ADF9BDE8BB
:109698000840054905480022FCF71CBD70BD0600BE
:1096A80048BD0600FFD80600B4C306000800002025
:1096B8002DE9F7439846174C174BDFF86C90E41ADE
:1096C800E408D9F800302404CDE9002305460B4608
:1096D8000E4617461149024644F00400FBF7A7F965
:1096E80029460F48CDF800803B463246FCF70AFD74
:1096F800054640B9D9F800300133C9F8003028468A
:1097080003B0BDE8F0830246064944F00200FBF7C7
:109718006FF9F4E770BD060048BD060027D90600BA
:10972800080000206AD90600CC1600202DE9F34174
:10973800134B144C144FE41AE4083B6800932404B8
:1097480005460B460E4690461049024644F0040072
:10975800FBF761F929460E4843463246FCF722FDDD
:10976800054630B93B6801333B60284602B0BDE886
:10977800F0810246074944F00200FBF739F9F4E7A3
:1097880048BD060070BD0600CC16002097D906001B
:1097980008000020D4D90600014B18700B20704730
:1097A800D0160020024B002218781A70704700BFAC
:1097B800D016002018DF704730B585B00546102256
:1097C8000C466846002102F032FAA4086846019562
:1097D8000294FFF7EFFF05B030BD30B585B0062322
:1097E80000244FF480556846CDE90035CDE90244A0
:1097F800FFF7E0FF072802BF4FF0005320461D6027
:1098080005B030BD084B09480949C01A10B5C00851
:10981800000440F00400FBF7E7F8064BBDE81040F1
:109828001B680620184700BF48BD060078BD060023
:109838000FDA0600DC1600200A2803D90B38C0B25C
:10984800FFF7AABF7047000070B5054686B0002034
:10985800FCF7E4FC0146A0B1274A18212846FCF78A
:1098680047F800283DD0254A254B26499B1ADB0896
:109878001B04024643F0010006B0BDE87040FBF748
:10988800B7B81822684602F0D2F904231C4C8DF8A8
:1098980000301A4B1C4EE41A1C4B1A6D3368E4084E
:1098A80024049A4244F004041DD119492046FBF7C8
:1098B8009BF8184B3168186801F028FE8DF80100F4
:1098C800FFF7BAFFD5E901138DF8010068469847FC
:1098D800114800F0A1FD9DF8012010492046FBF732
:1098E80087F806B070BD01238DF801306846D5E9C8
:1098F80001139847EFE700BF5198060048BD0600DE
:1099080078BD060043DA0600D4160020DC1F0020CC
:109918006CDA0600D81600200D9806009BDA0600BF
:109928002DE9F041836888B0044623B9A74940F27D
:10993800CF20FCF7C3F81822002102A802F077F91B
:10994800A34EA44B22788DF80820F61AF6080127B2
:1099580036048DF8097046F004050C2A00F24D8291
:10996800DFE812F00D00AE00A000AE00AE004B0222
:10997800AE009800AE00900026003D00A500964974
:109988002846FBF731F88DF80C709DF809209349AB
:109998002846FBF72DF8D4E9011302A898479DF84B
:1099A8000930012B00F013828D4B05201B680DE256
:1099B8008C492846FBF718F84FF08053D3F800215C
:1099C8000392D3F804210492D3F80C219202069250
:1099D800D3F81021920205921B690793D5E78249B3
:1099E800824E2846FBF700F8227C81492846FAF780
:1099F800FFFF4FF44053326A58687E49884214BFCB
:109A080001230223012A4FF001028DF80920227C4C
:109A180008BF013352B902238DF80C30F368049360
:109A2800754B0593C3F5FC230693AEE7012A12D1C3
:109A3800884210D100234FF440528DF80C30117831
:109A4800142988BF536904934FF4805305934FF446
:109A580040539B68E8E79A4209D201238DF80C30FD
:109A6800B368049300F016FEB3690590DCE7634918
:109A78002846FAF7B9FFFF238DF80C300023CDE90B
:109A88000433D1E75E492846FAF7AEFF237C8DF808
:109A98000C307AE75B492846FAF7A6FF238AADF827
:109AA8000C3072E758492846FAF79EFF6DE72846BA
:109AB8005649FAF799FF4A4B07201B68984764E70D
:109AC800062A534F01D0012A01D123693B703B7804
:109AD800012B0AD0022B00F0AF804E4946F001005E
:109AE800FAF782FF00233B7001E1013A072A66D8A2
:109AF800DFE802F004651444655D651E46492846A2
:109B0800FAF772FF364B03201B689847606901F02B
:109B1800B9F9FFF791FE8DF8090036E73F49284665
:109B2800FAF762FF314BDA6B1B6C039204932CE754
:109B3800236923B9254940F21310FBF7BFFFA38A15
:109B480023B922494FF48A70FBF7B8FF34492846F5
:109B5800FAF74AFFA18A206901F0ACF9FFF76CFE19
:109B6800224B8DF80900DA6B1B6C0493E3680392AF
:109B7800002B3FF40AAF2069984706E72949284691
:109B8800FAF732FF2849294801F012FAFFF754FE84
:109B980001288DF809007FF4F8AE002000F03CFCA5
:109BA80008B923497FE70A238DF80930EDE62149F2
:109BB8002846FAF719FF4FF400730593B2E70349F3
:109BC8004FF4BC70FBF77AFFDFE600BFC3DA06008C
:109BD80078BD060048BD060056DB06009BDA060085
:109BE800DC16002079DB06009CDB0600DC1F002069
:109BF800BFDB0600DBE5B15100400600DCDB0600F8
:109C0800F3DB06000ADC060024DC060048DC06005C
:109C180050000020E0DF060060DC06008ADC060059
:109C2800AEDC0600D7DC0600D4160020D8160020CB
:109C380002DD060027DD0600013A072A00F2D98076
:109C4800DFE812F00800D7009900A800D700C80084
:109C5800D70060006C492846FAF7C6FE01F05AF9A9
:109C680030B96A4946F00100FAF7BEFE08239BE7BF
:109C7800626932B9664946F00100FAF7B5FE032376
:109C880092E7C2F30B0343B1624B63495B6D09680A
:109C980013448B4201D06149EDE7B2F5805F06D9E4
:109CA8005F4946F00100FAF79FFE04237CE7594F0D
:109CB80059497B6D0968D018884206D9009146F049
:109CC80001005849FAF7A7FED0E77A64FA6CBA643B
:109CD800554A3B6510683B63002201211844FFF791
:109CE80025FD30B1514946F00100FAF77DFE052304
:109CF8005AE7BB6C00933B6D7A6C4D492846FAF7DE
:109D08008AFE42E64B492846FAF76EFE01F002F950
:109D18000028ABD03F4FA18AD7E914329B1A7A6C3E
:109D28000B44934201D94449A5E73F4A3B6B12686B
:109D3800206903EB020807F14802FBF7A3FEE3687A
:109D4800064623B93D494FF4F870FBF7B7FEE368C0
:109D5800A28A21694046FFF7ABFC08B1E3680AE72D
:109D6800A38A3A6BBE641A443A633A6D0496134464
:109D78003B65039309E6274E31492846FAF734FE36
:109D8800B36C326D2F492846FAF73BFEB36C049347
:109D9800336DEEE728462C49FAF726FE1D48D0E930
:109DA8001473426CFB1A934205D0284946F001000F
:109DB800FAF727FE5AE7836CC364002141644765BC
:109DC8002046FFF741FD224B1B680420984708B046
:109DD800BDE8F0811F492846FAF706FE0D4B4FF4FF
:109DE80080519A6C1B6D0591009104921A49039356
:109DF80084E7124940F29720E4E6184946F0030048
:109E0800FAF7F6FD0223CFE651DD060078DD0600FD
:109E1800ADDD0600DC1F0020D4160020C6DD0600DC
:109E2800E7DD06000BDE0600D81600207CDE060003
:109E380093DE0600CEDE0600F4DE0600C3DA060076
:109E48000BDF06002CDF060042DF06006ADF060093
:109E5800DC1600208EDF0600B5DF060000E00600F5
:109E6800836810B58BB10A4A1821FBF741FD0446F7
:109E780048B10848084B09491B1ADB081B0443F082
:109E88000200FAF7B1FD204610BD0724FBE700BF2A
:109E98002999060048BD060078BD06001FE00600A7
:109EA80038B50546C0B10020FFF7E6FB044648B9BF
:109EB80000F0DAFF01F02EF830B9084B00201D60E1
:109EC800FFF76AFC204638BD0549064801F070F8DE
:109ED8000128F2D00324F5E70724F3E7DC16002075
:109EE800D4160020D8160020011F0148FBF7B8BE81
:109EF800C4BD060013B5074C0A4601AB014620460F
:109F0800FCF7A4FC9DF8042003482146FDF734F82B
:109F180002B010BD7F1800205800002010B5064C74
:109F280023783BB1054B984204D00548FCF794FFD1
:109F380000232370002010BDE016002040BD06005D
:109F4800580000202DE9F047DFF8208198F800300C
:109F580088B00446002B62D1324B334E3349DFF8C8
:109F68001091F61AF608360446F0040A5046FAF735
:109F78003BFD2F48C9F80040FBF70CFE04460028BB
:109F880030D12B482B4F2C4DFBF742FE2B4B832215
:109F98000330C3E90104DA601C70294B7B60294B4C
:109FA800C7E90232284B3B61284B7B610FCD6C46D9
:109FB8000FC495E80F0084E80F0006220823CDE9B6
:109FC800002307210523CDE90213214A21480497DC
:109FD8006946FCF7C3FC044640B11F4946F001003E
:109FE800FAF702FD204608B0BDE8F0871B491C4877
:109FF8000122FDF739F8044620B11A4946F001005C
:10A00800FAF7F2FC50461849FAF7EEFCD9F8003096
:10A01800012088F80000002BE4D09847E2E70024EC
:10A02800E0E700BF48BD060088BD06004FE0060017
:10A03800C4BD0600B418002004E10600CC180020B6
:10A04800FD9E0600F19E06009818002040BD0600FF
:10A058007DA00600540000206BE00600B018002028
:10A068005800002084E006009BE00600E01600206F
:10A07800E416002070B50378012B0C4602D0022BA1
:10A0880033D070BD037A1BB343681A481978FCF7BC
:10A0980011FC0546184919480122FCF7E5FF002D77
:10A0A800EFD1144E2046D6E9011201F0C3FB144843
:10A0B800FBF7AEFD134B144A9B1ADB081B0404463E
:10A0C80040B9BDE87040114943F00100FAF78CBC73
:10A0D8000D25DFE702460E4943F003000334FAF783
:10A0E80087FCC6E901453570CBE7BDE87040C0681C
:10A0F800FDF7E0B9CC180020B01800205800002067
:10A10800C4BD060088BD060048BD0600C1E00600C3
:10A11800DBE006002DE9F74317464FF460729846D6
:10A128001F4D0646894601F022FD1E4BED1AED082B
:10A1380004462D0445F0040054B91B49FAF754FCB1
:10A148001FB9002003B0BDE8F0832046B847F8E700
:10A1580016490190FAF748FC154901983246FAF772
:10A1680047FC002201213046FFF7E0FA30B11149DF
:10A1780045F00100FAF738FC0320E3E74FF460727A
:10A188004946404601F02AFD3B464FF4607241467D
:10A198003046FFF78DFA0028D3D00749E8E700BF1B
:10A1A80090BD060048BD060024E106006EE10600E9
:10A1B80082E10600A2E10600C5E10600036801335A
:10A1C80010B5044609D0002258210430FBF75AFC88
:10A1D80023681B1A5842584110BD0020FCE70000B4
:10A1E8002DE9F0475048DFF87081504CDFF86C914A
:10A1F8004F4EFFF7E3FFD8F800A007465046FFF799
:10A20800DDFF0546002879D0DAF80450012D0AD080
:10A218000022C3210AF51870FBF734FCDAF85C5207
:10A228002B1A5D425D41002F58D0A4EB0907FF08A7
:10A238003F0447F004073F493846FAF7D5FB3A4947
:10A248003B484FF4607201F0C9FC8DB13A49384679
:10A25800FAF7CAFBD8F8005038485422291D01F0F3
:10A26800BDFC374840F2C72205F15C0101F0B6FC9D
:10A278007368012B55D1A4EB0900C00800043149CB
:10A2880040F00300FAF7B0FB2F4A02F2C71402F1BC
:10A298004005134603CBAB42206061601A4604F1C7
:10A2A8000804F6D1294B03F2C71203F118051C461E
:10A2B80003CCAC4210605160234602F10802F6D18B
:10A2C80020681060002386F86032012286F8E232A6
:10A2D800F36986F8A122C6F8A23220E085B1A4EB82
:10A2E8000900C00800041A4940F00300FAF77CFB93
:10A2F800D8F800100E484FF46072B7E7002F94D1D9
:10A30800A4EB0900C0080004124940F00200FAF763
:10A318006BFB07484FF46072002101F088FC0223B0
:10A328007360BDE8F08700BF00F0070090BD06002D
:10A33800DC1F0020ECE1060001E20600E01F00201F
:10A3480038200020E8E2060038210020782100208B
:10A358002BE2060084E206006000002048BD0600EB
:10A3680070B50C4C054600225821201DFBF78AFBCE
:10A3780000222060C32104F51870FBF783FB2A46EE
:10A38800C4F85C022146044B0448BDE87040FFF75E
:10A39800C1BE00BFDC1F00205C1C002000F00700CD
:10A3A800F8B5134B134C144FE41AE40824040D4673
:10A3B8003A681249064644F00300FAF719FB2846A2
:10A3C800FFF7FCFE20B90E494FF4C170FBF776FB8E
:10A3D80032460C4B38682946FFF79CFE024630B1DE
:10A3E80044F001000849BDE8F840FAF701BBF8BDA0
:10A3F80048BD060090BD06006000002014E306007A
:10A408003EE30600DC180020CEE306000149FFF712
:10A41800C7BF00BF00F0070038B505460020FFF7AA
:10A428009FFF044618B903492846FFF7B9FF20469D
:10A4380038BD00BFDC1F002037B5114B114C124945
:10A44800E41AE4082404054644F00400FAF7CCFAB8
:10A458002846FFF711F940B10C49024644F00100C3
:10A46800FAF7C6FA032003B030BD0190FFF7B8FE33
:10A478000198FFF7D1FF0028F5D005490246EDE71E
:10A4880048BD060090BD06000BE406002EE4060059
:10A4980059E4060008B50648064B0749C01AC00823
:10A4A800000440F00200FAF79FFA002008BD00BF40
:10A4B80090BD060048BD060093E4060010B5084CA0
:10A4C8004FF40072FF2104F15C0001F0B0FB202280
:10A4D800002104F1380001F0AAFB0023236310BD1A
:10A4E800DC1F00202DE9F843154B164CDFF864807B
:10A4F800154E1649E41AE408A6EB08062404F608E3
:10A5080044F00404074632462046FAF771FA4FF041
:10A518000009B14501D100250BE058F8393038461B
:10A528009847054640B1034609494A462046FAF786
:10A5380068FA2846BDE8F88309F10109E9E700BF90
:10A5480048BD060058BD060048BD0600BEE406002A
:10A55800E2E4060040BD06002DE9F843154B164C11
:10A56800164D174F1749E41AE4087F1B2404FF0807
:10A5780044F0040406463A462046FAF739FA4FF002
:10A58800000805F10409B84501D100250BE059F888
:10A59800383030469847054640B103460A49424696
:10A5A8002046FAF72EFA2846BDE8F88308F1010894
:10A5B800E9E700BF48BD060058BD060040BD0600DB
:10A5C80048BD06000EE5060033E50600034A0023F1
:10A5D8000360436083601363704700BFDC1F002083
:10A5E80008B54FF440535A68124B9A4220D1124989
:10A5F8000023042243F20400FFF75AF858B10F4B26
:10A608000F481049C01AC0080004BDE8084040F0CF
:10A618000100FAF7E9B90C4A136A4FF44051012BCB
:10A6280008BF1062936989680B44A3F5805393614E
:10A6380008BD00BFDBE5B1518CE7060048BD060048
:10A6480058BD06005DE50600DC1F00204FF44053AE
:10A65800074A5968914201BF986800F6FF7020F4D4
:10A668007F6020F00F0018BF4FF48050704700BF84
:10A67800DBE5B15108B5FFF7E9FF054B9B691844C5
:10A6880000F6FF7020F47F6020F00F0008BD00BFC7
:10A69800DC1F0020FFF7DABF4FF48050704700003E
:10A6A8002DE9F04F89B00646039207936E4A6F4B27
:10A6B80006919B1ADB081B0443F004046C490493BD
:10A6C8002046FAF791F96B49DFF8F881DFF8F8913D
:10A6D800DFF8F8A132462046FAF78AF9069B664960
:10A6E800002B0CBF42464A462046FAF781F9039BE5
:10A6F8006249002B0CBF42464A462046FAF778F9D1
:10A70800079B5F49002B0CBF42464A462046FAF792
:10A718006FF94FF440535B495A685B4B20469A42A5
:10A7280014BF42464A46FAF763F958492046FAF7F1
:10A738005BF9DAF81830DAF8202055492046FAF79C
:10A7480060F9DAF82430DAF82C2052492046FAF772
:10A7580058F94FF0000B5FFA8BF3BBF1010F01932F
:10A768004CD0022B59D0FFF785FF039B0546002BE1
:10A7780042D0DAF82020531E5A425A410292464FDC
:10A78800AF4203D24549B120FBF798F9069B4449EB
:10A798007F1BB74238BF01235A4620460593FAF774
:10A7A80027F940492A462046FAF722F93E49B74296
:10A7B8002CBF42464A462046FAF71AF9029B3B4903
:10A7C800002B0CBF42464A462046FAF711F9059B72
:10A7D8003749002B0CBF42464A462046FAF708F98B
:10A7E800059BFBB1029BEBB90BF1010BBBF1030F0E
:10A7F800B1D1B74225D217E0039ABFE7FFF726FF8A
:10A80800079B05463BB94FF440521F4B5268D21A7A
:10A8180018BF0122B2E75A46B0E7012302934FF46A
:10A828008055ACE7B74209D2049B224943F00200A5
:10A83800FAF7DAF8042009B0BDE8F08F019B022B83
:10A848000DD11D492046FAF7CFF8FFF7C9FE20467B
:10A858001A49FAF7C9F81A48FFF7B8FE02E0019B4F
:10A86800002BF4D10020E6E748BD060058BD0600DD
:10A878007EE506009CE50600BCE50600CDE5060081
:10A88800DBE50600F0E50600DBE5B15100E6060071
:10A898000FE606002FE60600001006004FE6060049
:10A8A800DCE60600E6E60600FBE6060010E7060022
:10A8B80023E7060034E7060060E7060079E70600AC
:10A8C800F41F0020B6E50600B1E50600DC1F0020F5
:10A8D8002DE9F04F4049414E8A6B414DDFF82891F0
:10A8E800DFF828A1DFF828B185B06F465C3138461B
:10A8F800FAF7B0FC97E80F004FF0000886E80F0061
:10A90800384BF3604FF447724146284689F8008077
:10A91800CAF80080CBF8008001F089F932492A464C
:10A928003046FAF734FF044650B93048304B3149C5
:10A93800C01AC008000440F00100FAF755F814E006
:10A9480099F80090B9F1000F04D095F86C312C7883
:10A95800A3B374B1264B25482749C01AC008000480
:10A9680040F00100FAF740F80024204605B0BDE8A1
:10A97800F08F95F87241002CF7D0DBF80020DAF858
:10A9880000103846FAF766FC97E80F0086E80F00D3
:10A998004FF4B272414605F5BA7001F048F917490B
:10A9A80005F5BA723046FAF7F2FE044680B90F4848
:10A9B8000F4B1349C01AC0080004BCE7002CD4D0C0
:10A9C800AC79002CD1D008350E4B4C461D60CCE735
:10A9D80005F5BA75F8E700BFDC1F0020A82600209F
:10A9E8008C230020A9AA0600E4D7060098BD06001B
:10A9F80048BD060090E70600BDE7060030D7060010
:10AA0800DCE7060064270020882300208423002038
:10AA18008023002010B590F8553013F0FB0F08D1B3
:10AA280090F864202AB1846E74B30C600124204627
:10AA380010BD13F0010403D090F8564004B1846DA2
:10AA48009B07F1D590F85C30002BEDD00F4B026ED0
:10AA5800C3F5FC239A4201D81444E5E70C490D4894
:10AA6800401AC00800040C4940F00100F9F7C9FF7A
:10AA78000424074B07480949C01AC008000440F0DD
:10AA88000100F9F7B1FFD2E70F24F2E70040060012
:10AA980048BD060098BD060018E8060035E806001F
:10AAA8005B68DA68134B9A4230B408D1124D2B68B0
:10AAB80013B9124C236823B1114B00221A7030BC11
:10AAC8007047D0E90131194413F9010B0028A1EBB3
:10AAD8000302F9DB2B600A4B0A4822600121197036
:10AAE800094B0A49C01AC008000430BC40F00400F1
:10AAF800F9F77EBF30D7060084230020802300208A
:10AB08008823002098BD060048BD060066E80600B8
:10AB180000B591B0FCF708FC18B10D49DB20FAF735
:10AB2800CDFF0C4920226846FCF74EFC0A490B4829
:10AB380040236A46FCF750FB18B10549E520FAF7AF
:10AB4800BDFF074B01221A7011B05DF804FB00BF6E
:10AB580083E80600D4CB0600B8260020CCC0060047
:10AB68005C2300202DE9F047A4B081460E46174625
:10AB7800984678222023002106A80493DDF8B0A087
:10AB880001F055F800230593424B1B780BB9FFF7EA
:10AB9800BFFF4148414C4249241AE408240444F0C8
:10ABA80003052846F9F720FF46B944F002003D495D
:10ABB800F9F71AFF132024B0BDE8F087B9F1000FA8
:10ABC80005D028463849F9F70FFF1620F3E737492B
:10ABD80052462846F9F70CFF04AB0193344B009317
:10ABE80034495346424606A8FCF784FB00284ED158
:10ABF800402F4CD1304B314606F140021F4651F8E8
:10AC0800040B43F8040B9142F9D12C492846F9F773
:10AC1800EBFE402628482021FCF7E3FB244A049B4E
:10AC28002749CDE9007605A8FCF7F2FA024640B3B9
:10AC3800244944F00100F9F7DBFE44F004002249FE
:10AC48000390F9F7D1FE32461B490398F9F70EFF36
:10AC58001E490398F9F7C8FEBDF810201449039857
:10AC6800F9F704FF1A490398F9F7BEFE1949039842
:10AC78003246F9F7FBFEF9F757FD0028FBD105200E
:10AC880099E728461449F9F7AFFE012093E70A200F
:10AC980091E700BF5C23002048BD060098BD060070
:10ACA80015E906003DE9060051E9060068E90600D5
:10ACB8000027002058CD06002027002083E9060041
:10ACC800B826002094E90600B6E90600C1E90600A6
:10ACD800C7E90600D4CB0600D3E906004FF4405379
:10ACE8001F4A5B68934213B538D000F500514C6891
:10ACF800A11A4C424C4193422DD100F500525168A3
:10AD0800994228D14FF4405316481978142982BF24
:10AD18005B691549B3FBF1F3117898BF0023142937
:10AD280082BF52691049B2FBF1F21049A0EB010051
:10AD380098BF00220E490092C00893424FEA004093
:10AD48000C4A40F0030018BF0A460B4914BF0124FF
:10AD58000024F9F760FE204602B010BD0024CAE7BF
:10AD6800DBE5B15198BD060040420F0048BD060022
:10AD7800E2E90600E8E90600EEE906002DE9F043FD
:10AD8800ABB006460F4690461C4678222023002189
:10AD98000CA8039300F04BFF294B1B780BB9FFF766
:10ADA800B7FE2CB13146202204A8FCF7F1FA04AE14
:10ADB800244B254C2549DFF8AC90E41AE408240418
:10ADC80044F0040543463A462846F9F71AFE03AB11
:10ADD80001933A461E49CDF8009043460CA8FCF76B
:10ADE80089FA024640B144F001001A49F9F700FE19
:10ADF80000202BB0BDE8F08320223146484600F001
:10AE0800B6FED8B1144944F00200F9F7EDFD134934
:10AE18002846F9F7E9FD202231462846F9F726FEAB
:10AE28000F492846F9F7E0FD202249462846F9F758
:10AE38001DFEF9F779FC0028FBD1DAE70120D8E7F5
:10AE48005C23002048BD060098BD06002EEA0600D7
:10AE580058CD060061EA060092EA0600ACEA060050
:10AE6800BEEA06005D23002008B5044B986B08B1C4
:10AE7800FFF72EFD024B187008BD00BFDC1F002035
:10AE88006027002010B5044658B1B0F5007F0AD8F5
:10AE9800064B00221A70FFF711FB054B01209C633B
:10AEA80010BD0320FCE70420FAE700BF602700205C
:10AEB800DC1F002070B5134C0646E06BA36B4218EC
:10AEC8009A420D460BD9104B10481149C01AC008B8
:10AED800000440F00100F9F787FD032070BD5C30E5
:10AEE8000A462044314600F079FEE36B04F1400243
:10AEF8002B4429463046E363FAF7C4FD2064012059
:10AF0800ECE700BFDC1F002048BD060098BD060026
:10AF1800CEEA0600014B1878704700BF6027002072
:10AF2800F0B51C4C94F86C2185B07AB394F8D8022B
:10AF3800B4F8DA2204F5377104F5B874164E174DD3
:10AF4800336800932B68FFF70DFE0128074605D1EB
:10AF5800201D00F0DFFA0128074614D01048114CD4
:10AF68001149241AE408240444F00200F9F73CFDCE
:10AF780044F004000D490390F9F736FD328829683A
:10AF88000398F9F773FD384605B0F0BD1146104631
:10AF98000434D3E78C23002080230020842300205E
:10AFA80048BD060098BD0600F1EA060007EB06005A
:10AFB800384BD3E90E329A422DE9F04106460D4648
:10AFC8000DD0354B35483649C01AC008000440F04A
:10AFD8000100F9F709FD08242046BDE8F081314F4A
:10AFE80097F80080B8F1000F09D0FFF743FB2E4B0C
:10AFF800306029461868BDE8F041FFF70BBDFFF740
:10B0080067FC00283AD0FFF78BFF0128C6F80080BC
:10B018000446C5F8008022D1DFF88C802946D8F88C
:10B028000000FFF7F7FC0128044618D1D8F80020E3
:10B038002868138A1BB15369003B18BF01230022FB
:10B048001146FFF72DFB154D134BED1AED082D0496
:10B0580040B1164945F00100F9F7C6FC0424FFF792
:10B068002DFAB9E7FFF706FB11493060024645F0B3
:10B078000400F9F7BDFC01233B70ADE7064B074818
:10B088000C49C01AC008000440F00100F9F7ACFCF4
:10B098000524A1E7DC1F002048BD060098BD060076
:10B0A80015EB0600602700206427002030EB06001F
:10B0B8004BEB060067EB060037B50D46044630B982
:10B0C800074901924FF42C70FAF7F8FC019A012312
:10B0D800294604F1720003B0BDE83040FFF74EBEC8
:10B0E80083E8060013B50446084623781146032B67
:10B0F8002CD8DFE803F01402161F0022D4F8014010
:10B10800FAF7C0FC84420AD01448154B1549C01AF6
:10B11800C0080004012240F00400F9F769FC01208E
:10B1280012E00A4600230146601C02B0BDE8104048
:10B13800FFF724BE034600914022611C0020FFF760
:10B1480011FD431E5842584102B010BD40F2D9309B
:10B158000549FAF7B3FC0020F6E700BF98BD0600E2
:10B1680048BD060084EB060083E806002DE9F0439D
:10B17800A3B005460E461446002178221F4604A8AF
:10B1880020239DF8AC800393DDF8A89000F04FFDD4
:10B1980041220021284600F04AFDB6F89430A34227
:10B1A80082BF442303FB046393F8968085F80080EC
:10B1B800B8F1030F38D8DFE808F009020F2C002295
:10B1C80049463846FAF75EFCC5F801004A46394652
:10B1D8002846FFF787FF19E003AB01936B1C009328
:10B1E80016494B463A4604A8FCF784F80028EDD0E7
:10B1F800FBF7B2F9124B1349024613481B1ADB0836
:10B208001B0443F00100F9F7F3FB002023B0BDE86D
:10B21800F08344214C4333199A34B3F898203119F8
:10B22800681C00F0DBFCD1E70548074B0749C01A4A
:10B23800C0080004424640F00100E4E758CD06008B
:10B2480098BD0600A7EB060048BD0600D8EB06002F
:10B258002DE9F0479D4B1C68A4B005468846174663
:10B268000A4601462046FFF727FF002800F00A811A
:10B2780094F85560002E44D14FF00109CDE90089BA
:10B288002B463246214613A8FFF770FF58B9002F06
:10B2980000F0F18005248E48FFF798F9FFF70EF9C2
:10B2A8008C4B9D64EAE0002F49D08A4F412213A9B4
:10B2B80007F2A12000F092FC874B88488849C7F81C
:10B2C8002C90C01AC008000440F00400F9F78CFB69
:10B2D800238A3E620BB163690BB9FFF781F994F8D1
:10B2E800923013B194F893300BB96368BB600022B5
:10B2F80041462846FAF7C6FB764B0124C3E9098084
:10B30800CCE74122002102A800F091FC06F0010AD6
:10B318004122002113A8D14606F0020600F087FC5E
:10B32800BAF1000F40F0B380002E40F09D806D49C7
:10B3380040F26130FAF7C2FB002F40F09880654B6D
:10B3480001245C619AE0A36D03F5FF5203F6FF73D5
:10B358001F32C3F30B03D31A82689A4206D25F489E
:10B368005D4B6149C01AC00800049DE04FF440538A
:10B378005A688A4215D11A78102A88BF1A6905F5C1
:10B38800005398BF0022197810298CBF1B6900232D
:10B398009A4206D05148504B5449C01AC00800047C
:10B3A80082E02846FFF79AFC48B14C484A4B50497E
:10B3B800C01AC008000440F00200F9F715FB012389
:10B3C8000193A36D009300222B46214602A8FFF7A4
:10B3D800CDFE00286CD0D6B1A26DAB18A8EB020246
:10B3E8000021CDE9002113A84A462146FFF7BEFEF9
:10B3F80000285DD09DF84C304BB13848364B3D495C
:10B40800C01AC008000440F00200F9F7EDFA002F56
:10B4180095D0B9F1000F2AD02846FFF75FFC10B18C
:10B428003548FFF7D3F84122344802A900F0D6FB8B
:10B43800284B002E14BFAC22A522DA62A26D5A63F3
:10B44800002E3FF454AF2E48412213A900F0C6FB4A
:10B4580094F8923023B194F89330002B7FF447AFDF
:10B468001C4B6268DA6042E742462B46B8E7194B44
:10B47800AA22DA62E4E70524FFF720F8204624B080
:10B48800BDE8F0871724002F7FF405AFF4E705F532
:10B4980000501C4B416899423FF455AF0F480E4B82
:10B4A8001949C01AC008000440F00100F9F79CFAD5
:10B4B800002FE0D0BAF1000F3FF4ECAEFFF7ECF844
:10B4C800A8427FF4E7AEFFF78BF8E3E66427002095
:10B4D80000200020DC1F002048BD060098BD0600A3
:10B4E800F9EB060083E8060072EC0600DBEC0600C8
:10B4F80048ED060089ED0600F41F00203C220020DC
:10B50800BE220020DBE5B15121EC06000122FFF745
:10B518009FBE0000F8B5044618B95449C420FAF78C
:10B52800CDFA94F854309BB194F8550003280FD8FD
:10B5380094F86E30032B17D04D4B4E484E49C01A25
:10B54800C008000440F00100F9F74EFA1420F8BDD5
:10B558004848474B4949C01AC008000440F0010058
:10B56800F9F742FA0F20F2E794F892301BB194F8F9
:10B578009330002B77D1237A33B93E483C4B40496E
:10B58800C01AC0080004E9E7E368342B0BD0384B35
:10B5980038483C49C01AC008000440F00200F9F7D6
:10B5A80023FA1120D3E74FF44051374A4D68238AD4
:10B5B80095423BD143B1626922B3DBB204F1140571
:10B5C8000022D6B2B3420BD8294B2A482F49C01AB9
:10B5D800C008000440F00200F9F706FA1220B6E7A6
:10B5E80055F8047B8E89B74202F10102E9D123782C
:10B5F8001BBB0128ABD01F481D4B2549C01AC008EA
:10B608000004ABE778B9012BF1D0DBB204F11405E3
:10B61800D6B2B342D8D955F8047B8E89B74202F125
:10B628000102F5D1E3E70128E1D1CDE713B1636960
:10B63800002BC9D12378002BC6D001286368154A8E
:10B648000ED8926893420ED2094B0A481249C01A82
:10B65800C008000440F00200F9F7C6F9102076E7A8
:10B66800D2689342F0D9012071E700BFE0ED0600EF
:10B6780048BD0600A0BD06008DEE060076EE060069
:10B68800A0EE0600AFEE0600DBE5B151C2EE060003
:10B69800E6EE0600DC1F0020D2EE0600030A087062
:10B6A8004B70030C000EC8708B70042070470000AC
:10B6B800F8B54278012A04460F4609D05748584B36
:10B6C8005849C01AC008000440F00200F9F790F980
:10B6D8002378082B0DD17B883A88013B9BB27B806D
:10B6E800002A00F09A80002B40F0978003237A808C
:10B6F80023704B4B494E3D6922784B49F61AF608A0
:10B708003604637846F00400F9F77BF960232B7060
:10B7180023786B706378AB70012B73D123780B2B74
:10B7280079D8DFE803F06B78784378784D5A786BEE
:10B738000630E91C6068FFF7B1FF0330C2B255FA62
:10B7480080F1A068FFF7AAFF1044C2B255FA80F151
:10B75800E068FFF7A3FF1044C2B255FA80F12069F0
:10B76800FFF79CFF1044C2B255FA80F16069FFF7F9
:10B7780095FF1044C4B2182C34D92C4946F0010066
:10B78800F9F732F92EE02379EB70291DA068FFF74D
:10B7980085FF0430C2B255FA80F1E068FFF77EFFFA
:10B7A8001044C2B255FA80F12069E0E76068E91CEC
:10B7B800FFF774FF0330C2B255FA80F1A068D6E7EC
:10B7C800E91CE068FFF76AFF0330C2B255FA80F15E
:10B7D8006068FFF763FF1044EDE7A388EB701B0A6E
:10B7E8002B7105247B68214628469847A8B146F066
:10B7F80001000F49BDE8F840F9F7F6B82379EB7076
:10B808000424EFE70B2B06D1FDF7CCFFE8700020EE
:10B81800FDF7C2FFF4E70324E4E7F8BD80BD0600A6
:10B8280048BD060011EF060039EF06005CEF060080
:10B838007DEF0600F0B50E4687B004460D46174664
:10B8480000211822684600F0F2F916F8013B394A3F
:10B858008DF800300B2B019402920BD863B1013B99
:10B868000A2B09D8DFE803F01F0C0808081C3D2C38
:10B878004B085600772B51D0A3683046984725E0EF
:10B888002D4B2E4822882E49C01AC008000440F0CB
:10B898000400F9F7ADF8B5F8013023806380EBE7D1
:10B8A8006B780493E8E7238863806B78D5F80220E7
:10B8B8000493012B0592DFD16069FEF74DFEDBE7AB
:10B8C800A3680496013FADF8147003936846FEF729
:10B8D800C7FA20B11B494FF48B70FAF7EFF807B09D
:10B8E800F0BD154B15481849C01AC008000440F0AF
:10B8F8000400F9F779F8E368ADF81030BCE70F48B1
:10B908000D4B6A781149C01AC008000440F00400C1
:10B91800F9F76EF86B788DF81030ADE7064B0748ED
:10B928006A780B49C01AC008000440F00400F9F70F
:10B938005FF8A1E7B9B6060048BD060080BD06005D
:10B94800A8EF0600FDEF0600C5EF0600D9EF0600D8
:10B95800EAEF06000369C26893429CBF80681B181F
:10B96800013B981A70472DE9F843D0E9029405463F
:10B97800A9EB04084068904520440F46144404D9B4
:10B9880000F02CF9EC60BDE8F8834246A4EB09040A
:10B9980000F024F96868224607EB0801F0E72DE972
:10B9A800F843C5680646894617464FF000083469CB
:10B9B800B3687068A54228BFE418013C621B5C1B91
:10B9C800BC4228BF3C46944228BF144649462844F6
:10B9D800224600F003F9B3682544AB4208BF0025AE
:10B9E8003F1BA044A144F560E1D14046BDE8F8837F
:10B9F80010B5114C114AA2610223C4E90433104B5B
:10BA0800E361A2644FF480530E4A0F492362E26453
:10BA180000231022E01DA3626362E362A3656365ED
:10BA2800E365226500F036F90849204600F032F94E
:10BA38002023A37110BD00BF68270020A1F00600D5
:10BA4800F0270020E0270020AAF00600AEF006004C
:10BA580070B5164B182400FB04451D4404FB003345
:10BA68001646DC6A012C0ED0022C18D0E4B9284600
:10BA7800FFF770FF864204D832462846FFF773FF67
:10BA88003446204670BD2846FFF764FF8642344698
:10BA980028BF044622462846FFF765FFF1E72846F7
:10BAA800BDE87040FFF77BBF0024EAE76827002065
:10BAB800FFF79EBF7F2805D8034B185C034B5B5CE0
:10BAC8001840704700207047C4F0060044F1060093
:10BAD800A0F16103192B98BF20387047A0F14103EA
:10BAE800192B98BF203070477F2805D8034B185C66
:10BAF800034B5B5C1840704700207047C4F0060099
:10BB080044F10600A0F16103192B98BF2038704753
:10BB1800A0F14103192B98BF203070477F299ABFA5
:10BB2800017001206FF02E0070475AB10A787F2A01
:10BB38000AD800B10260002119605960501A18BF74
:10BB480001207047002070476FF02E0070470000FA
:10BB580008B5034B5B689B681B68984708BD00BF26
:10BB68006400002008B50921FFF7F2FF08BD9AB369
:10BB780030B594460F2A18D902460B4640EA01040C
:10BB880014F0030F02D00CF1FF3C11E019461046E7
:10BB9800043204330C680568A54206D110461946DC
:10BBA800ACF1040CBCF1040FF0D8BCF1010C0FD0BF
:10BBB8000A46034684441146184601330132047884
:10BBC80091F800E0744503D1184611466345F2D157
:10BBD80000780B78C01A30BD00207047844640EAD0
:10BBE800010313F0030F18D18446202A0BD32DE943
:10BBF800F007B1E8F807A0E8F807A2F12002202A28
:10BC0800F7D2BDE8F007042A07D351F8043B40F8FF
:10BC1800043BA2F10402042AF7D2002A05D011F845
:10BC2800013B00F8013B013AF9D160467047844670
:10BC3800002A2DD010F0030F04D000F8011B013AA0
:10BC480026D0F7E7C9B241EA012141EA0141202A99
:10BC580012D3A2F120022DE9F0030B460C460D4643
:10BC68000E460F4688468946A0E8FA03203AFBD2DA
:10BC7800BDE8F00320320BD0042A05D340F8041B9A
:10BC8800043A05D0042AF9D200F8011B013AFBD185
:10BC980060467047024610F0030F16D111F0030FEB
:10BCA80013D12DE9F0004FF001374FF0803351F8F0
:10BCB800044BA4EB070525EA04051D4002D142F810
:10BCC800044BF4E7A1F10401F0BC11F8013B02F8C0
:10BCD800013B002BF9D1704700F1010110F0030F6F
:10BCE80011D010F8012B002A23D010F0030F0AD02E
:10BCF80010F8012B002A1CD010F0030F03D010F805
:10BD0800012B002A15D02DE970004FF001324FF0B9
:10BD1800803350F8044BA4EB020525EA04051D40C6
:10BD280000D1F6E7A0F1040070BC10F8012B002A3E
:08BD3800FBD1A0EB01007047F4
:08BD40004D9F0600259F06003F
:10BD480095CA06000000000044CB06000000000071
:10BD58004FBF06000000040483C106000000000075
:10BD680080D606000000040401DA0600000004047E
:10BD78003BE006000000040492F006000000040402
:10BD8800EFE0060000000404ADE40600000004042F
:10BD9800CDED060000000404FAEE060000000404DD
:08BDA8009BC306000000040427
:10BDB000BC000020840100208C010020C400002071
:10BDC00018000000E81600207C1800207F180020D2
:08BDD000F016002084000000C1
:10BDD80008BE060000000000A5BE06001C000020EA
:10BDE8000000000000000000F995060000100000A7
:04BDF800000008003F
:10BDFC00000000000338FDD870470000BD4306006A
:10BE0C0029440600B9430600443A5C576F726B5FD5
:10BE1C004A616B756A615C5355484F5F494D4147A8
:10BE2C00455C31315F454D455247454E43595F5353
:10BE3C0057495443485C23544F4F4C535C737263C3
:10BE4C005F32303231313232325C30335F6466759E
:10BE5C005F73657269616C2E32303231313232343B
:10BE6C005C636F6D706F6E656E74735C6C6962721F
:10BE7C0061726965735C6C6F675C7372635C6E7224
:10BE8C00665F6C6F675F64656661756C745F626139
:10BE9C00636B656E64732E63007274745F6C6F6792
:10BEAC005F6261636B656E6400443A5C576F726BE2
:10BEBC005F4A616B756A615C5355484F5F494D41F0
:10BECC0047455C31315F454D455247454E43595FBF
:10BEDC005357495443485C23544F4F4C535C737233
:10BEEC00635F32303231313232325C30335F646610
:10BEFC00755F73657269616C2E323032313132325A
:10BF0C00345C636F6D706F6E656E74735C6C6962BC
:10BF1C007261726965735C6C6F675C7372635C6E83
:10BF2C0072665F6C6F675F66726F6E74656E642E9F
:10BF3C0063004261636B656E647320666C75736835
:10BF4C006564006170700000AC1100207F0000007F
:10BF5C002C1200201B5B313B33316D0025734C6F71
:10BF6C0067732064726F70706564202825642925BE
:10BF7C00730D0A001B5B306D003C25733E2025734E
:10BF8C003A2000202530327800202020007C00252B
:10BF9C0063001B5B313B33306D001B5B313B333239
:10BFAC006D001B5B313B33336D001B5B313B33341A
:10BFBC006D001B5B313B33356D001B5B313B333606
:10BFCC006D001B5B313B33376D006572726F720015
:10BFDC007761726E696E6700696E666F0064656288
:10BFEC007567000080BF06009EBF060060BF06009C
:10BFFC00A6BF0600AEBF0600B6BF0600BEBF060059
:10C00C00C6BF0600CEBF060000000000D6BF06006B
:10C01C00DCBF0600E4BF0600E9BF06002E2E2F2E63
:10C02C002E2F2E2E2F2E2E2F2E2E2F6D6F64756CE5
:10C03C0065732F6E7266782F68616C2F6E72665FF7
:10C04C006770696F2E6800443A5C576F726B5F4A79
:10C05C00616B756A615C5355484F5F494D4147456B
:10C06C005C31315F454D455247454E43595F5357FF
:10C07C00495443485C23544F4F4C535C7372635F79
:10C08C0032303231313232325C30335F6466755F5C
:10C09C0073657269616C2E32303231313232345CFC
:10C0AC00636F6D706F6E656E74735C626F617264DA
:10C0BC00735C626F617264732E630011121314004F
:10C0CC004800280000204000358206002553060059
:10C0DC00CB5206001B5806008B580600AB580600C6
:10C0EC001B520600DD510600B75706000000000089
:10C0FC00443A5C576F726B5F4A616B756A615C5353
:10C10C0055484F5F494D4147455C31315F454D4581
:10C11C005247454E43595F5357495443485C235447
:10C12C004F4F4C535C7372635F3230323131323269
:10C13C00325C30335F6466755F73657269616C2E57
:10C14C0032303231313232345C636F6D706F6E6508
:10C15C006E74735C6C69627261726965735C757420
:10C16C00696C5C6170705F7574696C5F706C617424
:10C17C00666F726D2E63006D656D5F6D6E6772001C
:10C18C00443A5C576F726B5F4A616B756A615C53C2
:10C19C0055484F5F494D4147455C31315F454D45F1
:10C1AC005247454E43595F5357495443485C2354B7
:10C1BC004F4F4C535C7372635F32303231313232D9
:10C1CC00325C30335F6466755F73657269616C2EC7
:10C1DC0032303231313232345C636F6D706F6E6578
:10C1EC006E74735C6C69627261726965735C6261B6
:10C1FC006C6C6F635C6E72665F62616C6C6F632EED
:10C20C006300443A5C576F726B5F4A616B756A618D
:10C21C005C5355484F5F494D4147455C31315F4553
:10C22C004D455247454E43595F5357495443485C1B
:10C23C0023544F4F4C535C7372635F323032313145
:10C24C003232325C30335F6466755F73657269617C
:10C25C006C2E32303231313232345C657874657226
:10C26C006E616C5C667072696E74665C6E72665F31
:10C27C00667072696E74662E6300443A5C576F7216
:10C28C006B5F4A616B756A615C5355484F5F494DF2
:10C29C004147455C31315F454D455247454E435909
:10C2AC005F5357495443485C23544F4F4C535C7372
:10C2BC0072635F32303231313232325C30335F6430
:10C2CC0066755F73657269616C2E32303231313252
:10C2DC0032345C65787465726E616C5C6670726920
:10C2EC006E74665C6E72665F667072696E74665FA1
:10C2FC00666F726D61742E630030313233343536B3
:10C30C00373839414243444546443A5C576F726B67
:10C31C005F4A616B756A615C5355484F5F494D418B
:10C32C0047455C31315F454D455247454E43595F5A
:10C33C005357495443485C23544F4F4C535C7372CE
:10C34C00635F32303231313232325C30335F6466AB
:10C35C00755F73657269616C2E32303231313232F5
:10C36C00345C636F6D706F6E656E74735C6C696258
:10C37C007261726965735C6673746F726167655C18
:10C38C006E72665F6673746F726167652E63006EA2
:10C39C0072665F6673746F726167650000100000EF
:10C3AC0004000000010000006D62060091620600AE
:10C3BC00A1620600B1620600056306007962060000
:10C3CC007D62060081620600443A5C576F726B5FB7
:10C3DC004A616B756A615C5355484F5F494D4147E3
:10C3EC00455C31315F454D455247454E43595F538E
:10C3FC0057495443485C23544F4F4C535C737263FE
:10C40C005F32303231313232325C30335F646675D8
:10C41C005F73657269616C2E323032313132323475
:10C42C005C636F6D706F6E656E74735C6C69627259
:10C43C0061726965735C6D656D6F626A5C6E726664
:10C44C005F6D656D6F626A2E63004E52465F535589
:10C45C004343455353004E52465F4552524F525F31
:10C46C005356435F48414E444C45525F4D495353DC
:10C47C00494E47004E52465F4552524F525F534F02
:10C48C0046544445564943455F4E4F545F454E41D3
:10C49C00424C4544004E52465F4552524F525F4902
:10C4AC004E5445524E414C004E52465F4552524FEF
:10C4BC00525F4E4F5F4D454D004E52465F455252B6
:10C4CC004F525F4E4F545F464F554E44004E5246AE
:10C4DC005F4552524F525F4E4F545F535550504F21
:10C4EC0052544544004E52465F4552524F525F499A
:10C4FC004E56414C49445F504152414D004E5246BC
:10C50C005F4552524F525F494E56414C49445F531E
:10C51C0054415445004E52465F4552524F525F496A
:10C52C004E56414C49445F4C454E475448004E5280
:10C53C00465F4552524F525F494E56414C49445FFB
:10C54C00464C414753004E52465F4552524F525F44
:10C55C00494E56414C49445F44415441004E524669
:10C56C005F4552524F525F444154415F53495A45C3
:10C57C00004E52465F4552524F525F54494D454F03
:10C58C005554004E52465F4552524F525F4E554CD9
:10C59C004C004E52465F4552524F525F464F5242EC
:10C5AC00494444454E004E52465F4552524F525FED
:10C5BC00494E56414C49445F41444452004E524608
:10C5CC005F4552524F525F42555359004E52465F8F
:10C5DC004552524F525F4D4F44554C455F4E4F5450
:10C5EC005F494E495449414C495A4544004E5246C4
:10C5FC005F4552524F525F4D555445585F494E4915
:10C60C00545F4641494C4544004E52465F45525298
:10C61C004F525F4D555445585F4C4F434B5F46410D
:10C62C00494C4544004E52465F4552524F525F4D65
:10C63C00555445585F554E4C4F434B5F4641494C02
:10C64C004544004E52465F4552524F525F4D555431
:10C65C0045585F434F4E445F494E49545F464149EC
:10C66C004C4544004E52465F4552524F525F4D4F1F
:10C67C0044554C455F414C52454144595F494E49E4
:10C68C005449414C495A4544004E52465F4552521A
:10C69C004F525F53544F524147455F46554C4C00E7
:10C6AC004E52465F4552524F525F4150495F4E4F7A
:10C6BC00545F494D504C454D454E544544004E52E7
:10C6CC00465F4552524F525F464541545552455F65
:10C6DC004E4F545F454E41424C4544004E52465FCE
:10C6EC004552524F525F494F5F50454E44494E4759
:10C6FC00004E52465F4552524F525F4452565F5461
:10C70C0057495F4552525F4F56455252554E004E57
:10C71C0052465F4552524F525F4452565F545749EE
:10C72C005F4552525F414E41434B004E52465F456E
:10C73C0052524F525F4452565F5457495F455252C2
:10C74C005F444E41434B004E52465F4552524F524E
:10C75C005F424C455F495053505F52585F504B54A9
:10C76C005F5452554E4341544544004E52465F452A
:10C77C0052524F525F424C455F495053505F4348B1
:10C78C00414E4E454C5F414C52454144595F4558D2
:10C79C0049535453004E52465F4552524F525F42DA
:10C7AC004C455F495053505F4C494E4B5F44495385
:10C7BC00434F4E4E4543544544004E52465F4552FE
:10C7CC00524F525F424C455F495053505F50454564
:10C7DC00525F52454A454354454400556E6B6E6F4B
:10C7EC00776E206572726F7220636F646500000053
:10C7FC000000000056C406000100000062C40600E0
:10C80C000200000080C4060003000000A1C4060062
:10C81C0004000000B4C4060005000000C5C40600F6
:10C82C0006000000D9C4060007000000F1C4060091
:10C83C000800000009C506000900000021C506001B
:10C84C000A0000003AC506000B00000052C50600A5
:10C85C000C00000069C506000D0000007DC5060037
:10C86C000E0000008FC506000F0000009EC50600DC
:10C87C0010000000B2C5060011000000C9C506007A
:10C88C0080000000D8C5060081000000F9C5060034
:10C89C008200000015C606008300000031C60600A9
:10C8AC00840000004FC606008500000070C606001C
:10C8BC008600000095C6060090000000ACC606007D
:10C8CC0091000000CAC6060092000000E8C60600EF
:10C8DC0000820000FDC60600018200001BC7060096
:10C8EC000282000037C706000084000053C7060010
:10C8FC000184000077C7060002840000A1C706006F
:10C90C0003840000C6C70600982F8A4291443771F1
:10C91C00CFFBC0B5A5DBB5E95BC25639F111F159B6
:10C92C00A4823F92D55E1CAB98AA07D8015B8312F8
:10C93C00BE853124C37D0C55745DBE72FEB1DE80A4
:10C94C00A706DC9B74F19BC1C1699BE48647BEEFD3
:10C95C00C69DC10FCCA10C246F2CE92DAA84744A5E
:10C96C00DCA9B05CDA88F97652513E986DC631A8D4
:10C97C00C82703B0C77F59BFF30BE0C64791A7D5B3
:10C98C005163CA0667292914850AB72738211B2E3B
:10C99C00FC6D2C4D130D385354730A65BB0A6A7623
:10C9AC002EC9C281852C7292A1E8BFA24B661AA82F
:10C9BC00708B4BC2A3516CC719E892D1240699D63F
:10C9CC0085350EF470A06A1016C1A419086C371EB8
:10C9DC004C774827B5BCB034B30C1C394AAAD84E96
:10C9EC004FCA9C5BF36F2E68EE828F746F63A578D1
:10C9FC001478C8840802C78CFAFFBE90EB6C50A464
:10CA0C00F7A3F9BEF27871C6443A5C576F726B5F4C
:10CA1C004A616B756A615C5355484F5F494D41479C
:10CA2C00455C31315F454D455247454E43595F5347
:10CA3C0057495443485C23544F4F4C535C737263B7
:10CA4C005F32303231313232325C30335F64667592
:10CA5C005F73657269616C2E32303231313232342F
:10CA6C005C6D6F64756C65735C6E7266785C647219
:10CA7C0069766572735C7372635C7072735C6E72F0
:10CA8C0066785F7072732E630050525300443A5CA8
:10CA9C00576F726B5F4A616B756A615C5355484F97
:10CAAC005F494D4147455C31315F454D45524745E6
:10CABC004E43595F5357495443485C23544F4F4C92
:10CACC00535C7372635F32303231313232325C30EC
:10CADC00335F6466755F73657269616C2E323032D8
:10CAEC0031313232345C6D6F64756C65735C6E72AF
:10CAFC0066785C647269766572735C7372635C6E83
:10CB0C007266785F75617274652E63002E2E2F2EFF
:10CB1C002E2F2E2E2F2E2E2F2E2E2F696E746567F4
:10CB2C00726174696F6E2F6E7266782F6E72667892
:10CB3C005F676C75652E6800554152544500443A48
:10CB4C005C576F726B5F4A616B756A615C535548D9
:10CB5C004F5F494D4147455C31315F454D4552472B
:10CB6C00454E43595F5357495443485C23544F4FE8
:10CB7C004C535C7372635F32303231313232325C1F
:10CB8C0030335F6466755F73657269616C2E323029
:10CB9C003231313232345C636F6D706F6E656E742E
:10CBAC00735C6C69627261726965735C63727970D3
:10CBBC00746F5C6E72665F63727970746F5F7368AA
:10CBCC00617265642E6300001D85DB303598B4916D
:10CBDC00A49E842B8A8FAC713F6865700F349CBD0A
:10CBEC001C79B71000F1C9B563F941D170D673CE79
:10CBFC00DCF7EC487D99B0EF9297D28B1DD0FFDE1D
:10CC0C006A7C7ABF604DD71F52656365697665642F
:10CC1C002061206661756C74212069643A2030783B
:10CC2C00253038782C2070633A20307825303878CD
:10CC3C002C20696E666F3A20307825303878005297
:10CC4C006563656976656420616E206572726F72CA
:10CC5C003A203078253038782100496E7369646544
:10CC6C00206D61696E004166746572206D61696E3C
:10CC7C002C2073686F756C64206E6576657220620B
:10CC8C006520726561636865642E00000000000019
:10CC9C00000000000338FDD8704700000820000198
:10CCAC00FFFFFFFFFFFFFFFFFFFFFFFF0000000084
:10CCBC00000000000000000001000000FFFFFFFF6B
:10CCCC00512563FCC2CAB9F3849E17A7ADFAE6BC22
:10CCDC00FFFFFFFFFFFFFFFF00000000FFFFFFFF54
:10CCEC0096C298D84539A1F4A033EB2D817D0377FA
:10CCFC00F240A463E5E6BCF847422CE1F2D1176B95
:10CD0C00F551BF376840B6CBCE5E316B5733CE2B67
:10CD1C00169E0F7C4AEBE78E9B7F1AFEE242E34F96
:10CD2C004B60D2273E3CCE3BF6B053CCB0061D65D3
:10CD3C00BC86987655BDEBB3E7933AAAD835C65A5C
:10CD4C00FB7B06004D7D0600AD7D060027850600A9
:10CD5C0021850600018506002000000078000000F7
:10CD6C0000000000526573657474696E6720626F11
:10CD7C006F746C6F616465722E00496E61637469C7
:10CD8C00766974792074696D656F75742E00696E9F
:10CD9C00207765616B206E72665F6466755F696E85
:10CDAC0069745F7573657200496E206E72665F629E
:10CDBC006F6F746C6F616465725F696E6974004249
:10CDCC006F6F742076616C69646174696F6E206634
:10CDDC0061696C65642E204E6F2076616C696420ED
:10CDEC0061707020746F20626F6F742E00426F6FD1
:10CDFC00742076616C69646174696F6E2066616918
:10CE0C006C65642E20536F66744465766963652087
:10CE1C0069732070726573656E7420627574206915
:10CE2C006E76616C69642E00426F6F742076616C53
:10CE3C0069646174696F6E206661696C65642E202B
:10CE4C0041707020697320696E76616C69642E0084
:10CE5C004170702069732076616C6964004446559A
:10CE6C00206D6F6465206265636175736520617008
:10CE7C0070206973206E6F742076616C69642E006B
:10CE8C00444655206D6F64652072657175657374C9
:10CE9C0065642076696120627574746F6E2E00442F
:10CEAC004655206D6F646520726571756573746588
:10CEBC0064207669612047505245475245542E00F4
:10CECC00556E726561636861626C6500456E746570
:10CEDC0072206D61696E206C6F6F7000443A5C5704
:10CEEC006F726B5F4A616B756A615C5355484F5F3B
:10CEFC00494D4147455C31315F454D455247454EA3
:10CF0C0043595F5357495443485C23544F4F4C5338
:10CF1C005C7372635F32303231313232325C3033B7
:10CF2C005F6466755F73657269616C2E3230323185
:10CF3C00313232345C636F6D706F6E656E74735C1E
:10CF4C006C69627261726965735C626F6F746C6F2D
:10CF5C00616465725C6E72665F626F6F746C6F6138
:10CF6C006465722E630052756E6E696E67206E7208
:10CF7C00665F626F6F746C6F616465725F61707015
:10CF8C005F73746172742077697468206164647271
:10CF9C006573733A203078253038780044697361B2
:10CFAC00626C696E6720696E7465727275707473E9
:10CFBC002E204E5649432D3E494345525B305D3A37
:10CFCC002030782578004661696C65642072756E36
:10CFDC006E696E67206E72665F6466755F6D6272F5
:10CFEC005F6972715F666F72776172645F616464AE
:10CFFC00726573735F736574282900436F756C6475
:10D00C00206E6F742070726F7465637420626F6F22
:10D01C00746C6F6164657220616E642073657474E6
:10D02C00696E67732070616765732C203078257882
:10D03C002E00436F756C64206E6F742070726F7469
:10D04C0065637420536F667444657669636520610B
:10D05C006E64206170706C69636174696F6E2C20F2
:10D06C00307825782E00443A5C576F726B5F4A61BA
:10D07C006B756A615C5355484F5F494D4147455C40
:10D08C0031315F454D455247454E43595F535749E2
:10D09C005443485C23544F4F4C535C7372635F3260
:10D0AC00303231313232325C30335F6466755F73EB
:10D0BC00657269616C2E32303231313232345C63DC
:10D0CC006F6D706F6E656E74735C6C696272617299
:10D0DC006965735C626F6F746C6F616465725C6EB2
:10D0EC0072665F626F6F746C6F616465725F6170A2
:10D0FC00705F73746172745F66696E616C2E63002D
:10D10C0074696D65725F61637469766174652028FA
:10D11C00307825782900443A5C576F726B5F4A610E
:10D12C006B756A615C5355484F5F494D4147455C8F
:10D13C0031315F454D455247454E43595F53574931
:10D14C005443485C23544F4F4C535C7372635F32AF
:10D15C00303231313232325C30335F6466755F733A
:10D16C00657269616C2E32303231313232345C632B
:10D17C006F6D706F6E656E74735C6C6962726172E8
:10D18C006965735C626F6F746C6F616465725C6E01
:10D19C0072665F626F6F746C6F616465725F6466F8
:10D1AC00755F74696D6572732E630074696D657259
:10D1BC005F73746F70202830782578290074696D3E
:10D1CC0065725F66697265202830782578290000C1
:10D1DC00000000000338FDD8704756657269667907
:10D1EC00696E6720424C3A20416464723A20307870
:10D1FC00253038782C205372633A2030782530381B
:10D20C00782C204C656E3A20307825303878004EDA
:10D21C006F20626F6F746C6F6164657220636F70E6
:10D22C0079206E65656465642C20626F6F746C6F19
:10D23C00616465722075706461746520636F6D70D4
:10D24C006C6574652E00436F7079696E6720626F30
:10D25C006F746C6F616465723A205372633A20305C
:10D26C0078253038782C204C656E3A203078253073
:10D27C003878005265717565737420746F20636F14
:10D28C00707920424C206661696C6564004E6F2099
:10D29C00636F7079206E656564656400443A5C5711
:10D2AC006F726B5F4A616B756A615C5355484F5F77
:10D2BC00494D4147455C31315F454D455247454EDF
:10D2CC0043595F5357495443485C23544F4F4C5375
:10D2DC005C7372635F32303231313232325C3033F4
:10D2EC005F6466755F73657269616C2E32303231C2
:10D2FC00313232345C636F6D706F6E656E74735C5B
:10D30C006C69627261726965735C626F6F746C6F69
:10D31C00616465725C6E72665F626F6F746C6F6174
:10D32C006465725F66775F61637469766174696F57
:10D33C006E2E6300436F7079696E672030782578A4
:10D34C0020746F20307825782C2073697A653A2008
:10D35C0030782578004661696C656420746F20779D
:10D36C007269746520696D61676520636F70796996
:10D37C006E672070726F677265737320746F2073A1
:10D38C00657474696E677320706167652E00456EF5
:10D39C00746572206E72665F626F6F746C6F61641D
:10D3AC0065725F6466755F73645F636F6E74696EDC
:10D3BC00756500536F757263652061646472657383
:10D3CC007320646F6573206E6F7420636F6E74616D
:10D3DC00696E20612076616C696420536F667444B9
:10D3EC0065766963652E00534420616C72656164D7
:10D3FC007920636F70696564005570646174696E3F
:10D40C00672053442E204F6C642053442076657261
:10D41C003A2025642C204E6577207665723A2025BB
:10D42C0064004661696C656420746F20636F707969
:10D43C00206669726D776172652E00456E74657237
:10D44C00206E72665F626F6F746C6F616465725F81
:10D45C0066775F61637469766174650056616C69A7
:10D46C00642041707000456E746572206E72665F48
:10D47C006466755F6170705F636F6E74696E7565FD
:10D48C000053657474696E6720617070206173203D
:10D49C0076616C69640043524320636F6D707574E0
:10D4AC006174696F6E206661696C656420666F7269
:10D4BC0020636F70696564206170703A20737263C9
:10D4CC00206372633A203078253038782C207265CE
:10D4DC0073206372633A20307825303878005661B7
:10D4EC006C69642053440056616C696420424C00A2
:10D4FC0056616C6964205344202B20424C00456ECD
:10D50C00746572206E72665F6466755F73645F62C9
:10D51C006C5F636F6E74696E75650053442B424C7F
:10D52C003A20534420636F7079206661696C65649E
:10D53C000053442B424C3A20424C20636F707920AC
:10D54C006661696C6564004E6F206669726D776107
:10D55C00726520746F2061637469766174652E0046
:10D56C0041637469766174696F6E206661696C657C
:10D57C00642077697468206572726F72202564204C
:10D58C002862616E6B20636F64653A203078257871
:10D59C0029004120536F6674446576696365206881
:10D5AC006173206A757374206265656E20616374A3
:10D5BC006976617465642E2049742773206C696BDD
:10D5CC00656C79207468617420616E206170706C78
:10D5DC0069636174696F6E2077696C6C20636F6D21
:10D5EC006520696D6D6564696174656C7900436F64
:10D5FC00756C64206E6F7420777269746520736526
:10D60C007474696E67732E00496E7465726E616C0A
:10D61C0020666565640057445420656E61626C65D4
:10D62C0064204352563A2564207469636B7300532B
:10D63C0074617274696E6720612074696D65722003
:10D64C00282564207469636B732920666F722066C9
:10D65C00656564696E67207761746368646F672EB3
:10D66C0000574454206973206E6F7420656E61629C
:10D67C006C6564006E72665F626F6F746C6F616470
:10D68C0065725F7764740000000101000000010105
:10D69C00000000000100010000000000010000007B
:10D6AC000000000002000500010000004200000024
:10D6BC00000000000000000000000000000000005E
:10D6CC0000000000010011000100FFFF010000003C
:10D6DC0000000000020017000200FEFF64010000C1
:10D6EC0030D7060000000000000000000000000021
:10D6FC00000000000100010000000000010000001B
:10D70C0000000000020005000100000022000000E3
:10D71C0000000000000000000000000000000000FD
:10D72C0000000000010011000400FCFF04000000D8
:10D73C0000000000020011000400FCFF04000000C7
:10D74C0000000000030021000400FCFF0400100096
:10D75C0000000000040011000100FFFF01000000A8
:10D76C0000000000050011000200FEFF0400000094
:10D77C0000000000060011000400FCFF0400000083
:10D78C0000000000070011000400FCFF0400000072
:10D79C0000000000080017000200FEFF240000003B
:10D7AC0000D70600090010000100FFFF0100000077
:10D7BC00E0D706000A0027000200FEFF4400030029
:10D7CC00A0D60600000000000000000000000000D1
:10D7DC000000000000000000010017000400FCFF26
:10D7EC0068010000D0D60600020017000400FCFF00
:10D7FC00AC01000014D8060000000000000000007E
:10D80C000000000000000000010007000000000004
:10D81C0068010000D0D606000200010000000000E4
:10D82C0001000000000000000300050001000000E2
:10D83C00420000000000000000000000000000009A
:10D84C000000000000000000456E746572696E6790
:10D85C0020444655206D6F64652E00436F756C64D3
:10D86C00206E6F7420696E6974616C697A652044EE
:10D87C004655207472616E73706F72743A203078F2
:10D88C00253038780077726974650065726173654C
:10D89C0000466C6173682025732073756363657330
:10D8AC00733A20616464723D25702C2070656E643F
:10D8BC00696E6720256400466C61736820257320AF
:10D8CC006661696C6564202830782578293A206176
:10D8DC006464723D25702C206C656E3D3078257823
:10D8EC002062797465732C2070656E64696E672094
:10D8FC00256400496E697469616C697A696E672088
:10D90C006E72665F6673746F726167655F6E766D5B
:10D91C0063206261636B656E642E006E72665F6677
:10D92C0073746F726167655F77726974652861647F
:10D93C0064723D25702C207372633D25702C206C15
:10D94C00656E3D2564206279746573292C20717590
:10D95C006575652075736167653A202564006E7284
:10D96C00665F6673746F726167655F777269746501
:10D97C002829206661696C65642077697468206564
:10D98C0072726F7220307825782E006E72665F6628
:10D99C0073746F726167655F65726173652861642A
:10D9AC0064723D307825702C206C656E3D256420AA
:10D9BC007061676573292C207175657565207573A9
:10D9CC006167653A202564006E72665F6673746FDA
:10D9DC00726167655F65726173652829206661698C
:10D9EC006C65642077697468206572726F72203080
:10D9FC007825782E006E72665F6466755F666C6162
:10DA0C00736800416C6C20666C617368206F706584
:10DA1C00726174696F6E73206861766520636F6DD7
:10DA2C00706C657465642E2044465520636F6D7070
:10DA3C006C657465642E004661696C656420746F56
:10DA4C00207363686564756C65206F626A656374C6
:10DA5C0020657865637574653A20307825782E00DA
:10DA6C0057686F6C65206669726D776172652069A5
:10DA7C006D6167652072656365697665642E2050FB
:10DA8C006F737476616C69646174696E672E005291
:10DA9C006571756573742068616E646C696E67205E
:10DAAC00636F6D706C6574652E20526573756C7444
:10DABC003A203078257800443A5C576F726B5F4A95
:10DACC00616B756A615C5355484F5F494D414745E1
:10DADC005C31315F454D455247454E43595F535775
:10DAEC00495443485C23544F4F4C535C7372635FEF
:10DAFC0032303231313232325C30335F6466755FD2
:10DB0C0073657269616C2E32303231313232345C71
:10DB1C00636F6D706F6E656E74735C6C696272614D
:10DB2C00726965735C626F6F746C6F616465725C53
:10DB3C006466755C6E72665F6466755F7265715F54
:10DB4C0068616E646C65722E630048616E646C650E
:10DB5C00204E52465F4446555F4F505F50524F54D3
:10DB6C004F434F4C5F56455253494F4E0048616EE0
:10DB7C00646C65204E52465F4446555F4F505F487B
:10DB8C00415244574152455F56455253494F4E00FE
:10DB9C0048616E646C65204E52465F4446555F4F3B
:10DBAC00505F4649524D574152455F564552534975
:10DBBC004F4E004669726D7761726520696D6167C1
:10DBCC0065207265717565737465643A202564000F
:10DBDC004E6F2073756368206669726D776172652C
:10DBEC0020696D6167650048616E646C65204E52FA
:10DBFC00465F4446555F4F505F50494E4700486161
:10DC0C006E646C65204E52465F4446555F4F505FC4
:10DC1C004D54555F4745540048616E646C65204E09
:10DC2C0052465F4446555F4F505F524543454950FD
:10DC3C00545F4E4F5449465F5345540048616E64DF
:10DC4C006C65204E52465F4446555F4F505F4142D3
:10DC5C004F52540048616E646C65204E52465F44CE
:10DC6C0046555F4F505F4F424A4543545F435245C0
:10DC7C004154452028636F6D6D616E6429004861C5
:10DC8C006E646C65204E52465F4446555F4F505F44
:10DC9C004352435F4745542028636F6D6D616E643A
:10DCAC00290048616E646C65204E52465F444655AF
:10DCBC005F4F505F4F424A4543545F57524954455A
:10DCCC002028636F6D6D616E64290048616E646C11
:10DCDC0065204E52465F4446555F4F505F4F424A57
:10DCEC004543545F455845435554452028636F6D53
:10DCFC006D616E64290057726974696E6720766174
:10DD0C006C696420696E697420636F6D6D616E64FB
:10DD1C0020746F20666C6173682E0048616E646CB1
:10DD2C0065204E52465F4446555F4F505F4F424A06
:10DD3C004543545F53454C4543542028636F6D6DE8
:10DD4C00616E64290048616E646C65204E52465FBA
:10DD5C004446555F4F505F4F424A4543545F4352D0
:10DD6C0045415445202864617461290043616E6EFD
:10DD7C006F74206372656174652064617461206FD7
:10DD8C00626A65637420776974686F757420766154
:10DD9C006C696420696E697420636F6D6D616E646B
:10DDAC00004F626A6563742073697A652063616EE3
:10DDBC006E6F7420626520302E004F626A6563744A
:10DDCC002073697A65206D757374206265207061AB
:10DDDC00676520616C69676E656400496E76616C7D
:10DDEC0069642073697A6520666F72206F626A6558
:10DDFC0063742028746F6F206C617267652900430F
:10DE0C0072656174696E6720746865206F626A65FB
:10DE1C00637420776974682073697A65203078257B
:10DE2C0030387820776F756C64206F766572666C0D
:10DE3C006F77206669726D776172652073697A6598
:10DE4C002E204F66667365742069732030782530F8
:10DE5C00387820616E64206669726D776172652016
:10DE6C0073697A65206973203078253038782E00F4
:10DE7C004572617365206F7065726174696F6E2095
:10DE8C006661696C6564004372656174696E6720D4
:10DE9C006F626A65637420776974682073697A6548
:10DEAC003A2025642E204F66667365743A203078CC
:10DEBC00253038782C204352433A2030782530389E
:10DECC00780048616E646C65204E52465F4446553E
:10DEDC005F4F505F4F424A4543545F575249544538
:10DEEC002028646174612900577269746520726519
:10DEFC00717565737420746F6F206C6F6E6700485A
:10DF0C00616E646C65204E52465F4446555F4F50BF
:10DF1C005F4352435F474554202864617461290074
:10DF2C004F66667365743A25642C204352433A302D
:10DF3C0078253038780048616E646C65204E524606
:10DF4C005F4446555F4F505F4F424A4543545F45CF
:10DF5C005845435554452028646174612900496E25
:10DF6C0076616C696420646174612E2065787065DB
:10DF7C00637465643A2025642C20676F743A2025FD
:10DF8C00640048616E646C65204E52465F44465591
:10DF9C005F4F505F4F424A4543545F53454C454396
:10DFAC00542028646174612900637263203D203021
:10DFBC007825782C206F6666736574203D20307848
:10DFCC0025782C206D61785F73697A65203D20304F
:10DFDC0078257800496E76616C6964206F626A6599
:10DFEC006374207479706520696E20726571756533
:10DFFC0073742E00496E76616C6964206F70636F68
:10E00C0064652072656365697665643A20307825AD
:10E01C00782E005363686564756C65722072616E4E
:10E02C00206F7574206F6620737061636521006EBC
:10E03C0072665F6466755F7265715F68616E646C51
:10E04C0065720073657269616C5F6466755F74728A
:10E05C00616E73706F72745F696E69742829004603
:10E06C0061696C656420696E697469616C697A694F
:10E07C006E672075617274004661696C6564206915
:10E08C006E697469616C697A696E67207278007365
:10E09C00657269616C5F6466755F7472616E7370D2
:10E0AC006F72745F696E6974282920636F6D706C70
:10E0BC0065746564004661696C656420746F2061E9
:10E0CC006C6C6F6361746520627566666572004185
:10E0DC006C6C6F6361746564206275666665722032
:10E0EC002578006E72665F6466755F736572696130
:10E0FC006C5F756172740000FFFFFFFFFFFFFFFF95
:10E10C00FFFFFFFFFFFFFFFF00000000000000000B
:10E11C000000D6010600000044657374696E6174DA
:10E12C00696F6E2073657474696E677320617265B4
:10E13C00206964656E746963616C20746F20736F01
:10E14C00757263652C207772697465206E6F74200C
:10E15C006E65656465642E20536B697070696E67BB
:10E16C002E0057726974696E672073657474696EDA
:10E17C0067732E2E2E0045726173696E67206F6C6B
:10E18C00642073657474696E67732061743A20300F
:10E19C00782530387800436F756C64206E6F74206E
:10E1AC006572617365207468652073657474696E3B
:10E1BC00677320706167652100436F756C64206E16
:10E1CC006F742077726974652074686520444655B5
:10E1DC002073657474696E677320706167652100C4
:10E1EC005573696E672073657474696E67732070FC
:10E1FC006167652E00436F7079696E6720666F7278
:10E20C0062696464656E2070617274732066726FEB
:10E21C006D206261636B757020706167652E0052B2
:10E22C006573746F72696E672073657474696E6759
:10E23C00732066726F6D206261636B7570207369F9
:10E24C006E6365207468652073657474696E67739A
:10E25C00207061676520636F6E74656E74732061E6
:10E26C00726520696E76616C696420284352432084
:10E27C006572726F72292E00526573657474696EC3
:10E28C006720626F6F746C6F616465722073657464
:10E29C0074696E67732073696E6365206E6569744B
:10E2AC00686572207468652073657474696E677331
:10E2BC002070616765206E6F7220746865206261E2
:10E2CC00636B7570206172652076616C69642028BF
:10E2DC00435243206572726F72292E004F6C64207A
:10E2EC0073657474696E677320706167652064650B
:10E2FC007465637465642E20557067726164696E11
:10E30C006720696E666F2E004261636B696E6720D1
:10E31C0075702073657474696E67732070616765BE
:10E32C0020746F2061646472657373203078257873
:10E33C002E00443A5C576F726B5F4A616B756A6171
:10E34C005C5355484F5F494D4147455C31315F4502
:10E35C004D455247454E43595F5357495443485CCA
:10E36C0023544F4F4C535C7372635F3230323131F4
:10E37C003232325C30335F6466755F73657269612B
:10E38C006C2E32303231313232345C636F6D706FDF
:10E39C006E656E74735C6C69627261726965735CD4
:10E3AC00626F6F746C6F616465725C6466755C6ED1
:10E3BC0072665F6466755F73657474696E67732EDD
:10E3CC006300436F756C64206E6F742070657266A9
:10E3DC006F726D206261636B7570206F6620626F67
:10E3EC006F746C6F616465722073657474696E67A9
:10E3FC007321204572726F723A2030782578004371
:10E40C00616C6C696E67206E72665F6466755F73B3
:10E41C00657474696E67735F696E697428292E2E32
:10E42C002E006E72665F6466755F666C6173685F02
:10E43C00696E69742829206661696C656420776946
:10E44C007468206572726F723A202578006E72665D
:10E45C005F6466755F73657474696E67735F7772FA
:10E46C006974655F616E645F6261636B75702829A6
:10E47C00206661696C6564207769746820657272C6
:10E48C006F723A202578004E6F206164646974695C
:10E49C006F6E616C20646174612065726173656478
:10E4AC00006E72665F6466755F73657474696E671F
:10E4BC007300496E697469616C697A696E6720745E
:10E4CC0072616E73706F7274732028666F756E64F0
:10E4DC003A20256429004661696C656420746F20BC
:10E4EC00696E697469616C697A65207472616E73A6
:10E4FC00706F72742025642C206572726F722025E7
:10E50C0064005368757474696E6720646F776E204D
:10E51C007472616E73706F7274732028666F756E8F
:10E52C00643A20256429004661696C656420746F27
:10E53C002073687574646F776E207472616E73707B
:10E54C006F72742025642C206572726F72202564A2
:10E55C0000436F756C64206E6F7420696E76616C0D
:10E56C00696461746520536F66744465766963658C
:10E57C002E00456E746572206E72665F6466755F00
:10E58C0063616368655F70726570617265282900EC
:10E59C0072657175697265645F73697A653A20306A
:10E5AC007825782E00747275650066616C73650051
:10E5BC0073696E676C655F62616E6B3A2025732EB2
:10E5CC00006B6565705F6170703A2025732E006B6F
:10E5DC006565705F736F66746465766963653A2010
:10E5EC0025732E0053445F50524553454E543A20E8
:10E5FC0025732E0042616E6B20636F6E74656E74B2
:10E60C00733A0042616E6B203020636F64653A2070
:10E61C003078253032783A2053697A653A20307850
:10E62C0025780042616E6B203120636F64653A205F
:10E63C003078253032783A2053697A653A20307830
:10E64C00257800443A5C576F726B5F4A616B756A50
:10E65C00615C5355484F5F494D4147455C31315FD3
:10E66C00454D455247454E43595F535749544348CE
:10E67C005C23544F4F4C535C7372635F32303231B6
:10E68C00313232325C30335F6466755F7365726948
:10E69C00616C2E32303231313232345C636F6D70DA
:10E6AC006F6E656E74735C6C6962726172696573AE
:10E6BC005C626F6F746C6F616465725C6466755CD0
:10E6CC006E72665F6466755F7574696C732E630039
:10E6DC00706173733A2025642E0063616368655F13
:10E6EC00616464726573733A20307825782E006308
:10E6FC00616368655F746F6F5F736D616C6C3A20FA
:10E70C0025732E006B6565705F6669726D7761723B
:10E71C00653A2025732E0064656C6574655F6D6FBA
:10E72C0072653A2025732E0041626F7274696E67B0
:10E73C002E2043616E6E6F7420666974206E65774F
:10E74C00206669726D77617265206F6E20646576E4
:10E75C0069636500496E76616C69646174696E67A2
:10E76C0020536F66744465766963652E00496E7636
:10E77C00616C69646174696E67206170702E000051
:10E78C000000000048616E646C65723A20496E7638
:10E79C00616C69642070726F746F636F6C2062754A
:10E7AC0066666572206D5F70625F73747265616D11
:10E7BC000048616E646C65723A20496E76616C69D2
:10E7CC006420696E697420636F6D6D616E642E00D8
:10E7DC0048616E646C65723A20496E76616C69644E
:10E7EC002070726F746F636F6C20627566666572F1
:10E7FC00206D5F70625F73747265616D2028696E45
:10E80C00697420636F6D6D616E642900424C2073D6
:10E81C00697A652028256429206F766572206C69D9
:10E82C006D6974202825642900496E697420706113
:10E83C00636B657420646F6573206E6F7420636FF7
:10E84C006E7461696E2076616C6964206669726DA4
:10E85C00776172652073697A650050423A20496E7F
:10E86C006974207061636B65742064617461206CE1
:10E87C00656E3A20256400443A5C576F726B5F4AB0
:10E88C00616B756A615C5355484F5F494D41474513
:10E89C005C31315F454D455247454E43595F5357A7
:10E8AC00495443485C23544F4F4C535C7372635F21
:10E8BC0032303231313232325C30335F6466755F04
:10E8CC0073657269616C2E32303231313232345CA4
:10E8DC00636F6D706F6E656E74735C6C6962726180
:10E8EC00726965735C626F6F746C6F616465725C86
:10E8FC006466755C6E72665F6466755F76616C6982
:10E90C00646174696F6E2E63005369676E61747510
:10E91C0072652072657175697265642E2043686535
:10E92C00636B696E67207369676E61747572652EAF
:10E93C00004E6F207369676E617475726520666F27
:10E94C00756E642E00496E76616C6964207369671C
:10E95C006E617475726520747970650043616C63C7
:10E96C00756C6174696E67206861736820286C65CA
:10E97C006E3A2025642900566572696679207369A0
:10E98C00676E6174757265005369676E6174757238
:10E99C0065206661696C656420286572725F636FBF
:10E9AC0064653A203078257829005369676E617464
:10E9BC007572653A00486173683A005075626C690B
:10E9CC0063204B65793A00496D6167652076657205
:10E9DC006966696564006D616A6F72006D696E6F5E
:10E9EC007200536F66744465766963652075706454
:10E9FC0061746520697320612025732076657273BC
:10EA0C00696F6E207570646174652E204375727227
:10EA1C00656E743A2025642E204E65773A20256465
:10EA2C002E0048617368207665726966696361744B
:10EA3C00696F6E2E207374617274206164647265E8
:10EA4C0073733A20307825782C2073697A653A20D4
:10EA5C003078257800436F756C64206E6F7420726B
:10EA6C00756E20686173682076657269666963618A
:10EA7C0074696F6E20286572725F636F64652030F5
:10EA8C00782578292E00486173682076657269664E
:10EA9C0069636174696F6E206661696C65642E00D0
:10EAAC0045787065637465642046572068617368A7
:10EABC003A0041637475616C204657206861736835
:10EACC003A00496E697420636F6D6D616E64206CE1
:10EADC006172676572207468616E20657870656319
:10EAEC007465642E0050726576616C69646174693A
:10EAFC006F6E206661696C65642E00496E697420C6
:10EB0C00636F6D6D616E643A00457865637574650D
:10EB1C002077697468206661756C7479206F6666FD
:10EB2C007365740043616E27742066696E6420728D
:10EB3C006F6F6D20666F722075706461746500571D
:10EB4C007269746520616464726573732073657493
:10EB5C0020746F20307825303878004661696C65F8
:10EB6C006420746F206465636F646520696E6974DA
:10EB7C00207061636B657400435243206368656366
:10EB8C006B206F6620617070206661696C65642E05
:10EB9C002052657475726E202564006E72665F6318
:10EBAC00727970746F5F686173685F63616C6375B1
:10EBBC006C6174652829206661696C6564207769CD
:10EBCC007468206572726F7220257300496E7661CD
:10EBDC006C696420626F6F742076616C6964617417
:10EBEC00696F6E20747970653A20256400496E76E1
:10EBFC00616C69646174696E67206F6C642061700C
:10EC0C00706C69636174696F6E20696E2062616EED
:10EC1C006B20302E0054686520536F667444657603
:10EC2C0069636520646F6573206E6F7420636F6E0B
:10EC3C007461696E20746865206D61676963206E0C
:10EC4C00756D626572206964656E74696679696E4A
:10EC5C0067206974206173206120536F667444656A
:10EC6C00766963652E0054686520536F667444653D
:10EC7C00766963652073697A6520696E20746865AE
:10EC8C0020696E666F2073747275637420697320CB
:10EC9C00746F6F20736D616C6C20636F6D7061723B
:10ECAC0065642077697468207468652073697A6577
:10ECBC00207265706F7274656420696E207468656B
:10ECCC0020696E697420636F6D6D616E642E0054E3
:10ECDC006865206E657720536F667444657669634A
:10ECEC0065206973206F66206120646966666572B1
:10ECFC00656E742066616D696C79207468616E2034
:10ED0C007468652070726573656E7420536F6674D9
:10ED1C004465766963652E20436F6D70617469621A
:10ED2C00696C6974792063616E6E6F742062652002
:10ED3C0067756172616E746565642E00496E7661EB
:10ED4C006C69646174696E672061707020626563C0
:10ED5C006175736520697420697320696E636F6DCA
:10ED6C0070617469626C6520776974682074686579
:10ED7C0020536F66744465766963652E00426F6F2D
:10ED8C00742076616C69646174696F6E206F6620A3
:10ED9C00626F6F746C6F61646572206973206E6F43
:10EDAC007420737570706F7274656420616E64206A
:10EDBC0077696C6C2062652069676E6F7265642E72
:10EDCC00006E72665F6466755F76616C696461740F
:10EDDC00696F6E00443A5C576F726B5F4A616B757A
:10EDEC006A615C5355484F5F494D4147455C313131
:10EDFC005F454D455247454E43595F535749544320
:10EE0C00485C23544F4F4C535C7372635F32303207
:10EE1C0031313232325C30335F6466755F736572E8
:10EE2C0069616C2E32303231313232345C636F6D49
:10EE3C00706F6E656E74735C6C6962726172696519
:10EE4C00735C626F6F746C6F616465725C64667521
:10EE5C005C6E72665F6466755F7665725F76616C18
:10EE6C0069646174696F6E2E6300496E76616C69BA
:10EE7C0064206669726D7761726520747970652E95
:10EE8C0000496E76616C69642068617368207479DE
:10EE9C0070652E004E6F2048572076657273696F2F
:10EEAC006E2E004661756C74792048572076657219
:10EEBC0073696F6E2E00534420726571206E6F74EF
:10EECC00206D65742E0046572076657273696F6EDF
:10EEDC0020746F6F206C6F772E004657207665720A
:10EEEC0073696F6E206D697373696E672E006E7235
:10EEFC00665F6466755F7665725F76616C69646186
:10EF0C0074696F6E00444655207265717565737433
:10EF1C0020636F6D706C657465642077697468200C
:10EF2C00726573756C743A20307825780053656E71
:10EF3C0064696E6720526573706F6E73653A205BFF
:10EF4C003078253031782C203078253031785D00C0
:10EF5C004D657373616765206973206C61726765B9
:10EF6C0072207468616E2065787065637465642EB8
:10EF7C00004661696C656420746F2073656E642053
:10EF8C0064617461206F7665722073657269616C5F
:10EF9C0020696E7465726661636521005365742027
:10EFAC0072656365697074206E6F74696620746134
:10EFBC00726765743A2025640052656365697665ED
:10EFCC00642073657269616C206D747500526563A1
:10EFDC0065697665642070696E67202564005265EA
:10EFEC006365697665642055706461746520256479
:10EFFC0000443A5C576F726B5F4A616B756A615C77
:10F00C005355484F5F494D4147455C31315F454D44
:10F01C00455247454E43595F5357495443485C2327
:10F02C00544F4F4C535C7372635F32303231313218
:10F03C0032325C30335F6466755F73657269616C24
:10F04C002E32303231313232345C636F6D706F6E10
:10F05C00656E74735C6C69627261726965735C6213
:10F06C006F6F746C6F616465725C73657269616CEF
:10F07C005F6466755C6E72665F6466755F736572FD
:10F08C0069616C2E63006E72665F6466755F736592
:10F09C007269616C005465726D696E616C005254DA
:10F0AC005400534547474552000000004300000000
:10F0BC00504F5349580000002020202020202020B1
:10F0CC0020682828282820202020202020202020CC
:10F0DC00202020202020202048101010101010106C
:10F0EC001010101010101010848484848484848474
:10F0FC008484101010101010108181818181810185
:10F10C0001010101010101010101010101010101E3
:10F11C000101011010101010108282828282820272
:10F12C0002020202020202020202020202020202B3
:10F13C000202021010101020000703200417020115
:10F14C000857104080000000B8F00600BCF1060023
:10F15C00D0F2060053756E004D6F6E00547565004D
:10F16C0057656400546875004672690053617400F9
:10F17C00000000004A616E00466562004D6172003D
:10F18C00417072004D6179004A756E004A756C00D1
:10F19C0041756700536570004F6374004E6F7600C5
:10F1AC004465630000000000414D00504D0000001C
:10F1BC00F4F20600F0F20600F0F20600F0F206009F
:10F1CC00F0F20600F0F20600F0F20600F0F2060093
:10F1DC00F0F20600F0F20600FFFFFFFFFFFFFFFF5B
:10F1EC00FFFFFFFFFFFF000030F2060060F106009A
:10F1FC006CF2060080F10600B4F1060014F2060071
:10F20C00C4F2060020F20600256D2F25642F257907
:10F21C000000000025612025622025652025542052
:10F22C002559000053756E646179004D6F6E6461F1
:10F23C00790054756573646179005765646E657304
:10F24C0064617900546875727364617900467269FF
:10F25C006461790053617475726461790000000017
:10F26C004A616E7561727900466562727561727978
:10F27C00004D6172636800417072696C004D617978
:10F28C00004A756E65004A756C7900417567757337
:10F29C00740053657074656D626572004F63746FB2
:10F2AC00626572004E6F76656D62657200446563CF
:10F2BC00656D62657200000025483A254D3A25536C
:10F2CC0000000000BDBA0600D9BA0600E5BA060077
:10F2DC00F1BA06000DBB060019BB060025BB0600E3
:0AF2EC0033BB0600000000002E00F6
:10F2F80000000000FF000000000000000000000007
:10F3080000000000000000000000000000000000F5
:10F31800000000000100000024000020340000204C
:10F328000090D00301000000000000000020004011
:10F338000000000000E0070054F1060054F1060048
:0CF3480054F1060054F1060054F10600D8
:020000020000FC
:020000041000EA
:041014000040060092
:0410180000E00700ED
:040000036000435DF9
:00000001FF
